:100000000C94CE030C94EB030C9414250C94EB038A
:100010000C94EB030C94EB030C94EB030C94EB03A8
:100020000C94EB030C94DC3A0C94EB030C94EB0370
:100030000C94EB030C94EB030C94EB030C94EB0388
:100040000C94EB030C94EB030C94EB030C94EB0378
:100050000C94EB030C9466480C94EB030C94EB03A8
:100060000C94EB030C94EB030C94EB030C94EB0358
:100070000C94EB030C94EB030C94EB030C94EB0348
:100080000C94EB030C94EB030C94EB030C94EB0338
:100090000C94EB03613CAC3C6B3D913D083E2B3E28
:1000A0004F3E523E613ECE45CE45CE45CE45CE4535
:1000B000CE45CE45CE45CE45CE45CE45CE45CE45A8
:1000C000CE45CE45CE45CE45CE45CE45CE45CE4598
:1000D000CE45EE3E703E8B3E0C3F1C3F9040C840EC
:1000E0000D414F418B41FE41CE45CE45CE45CE45DB
:1000F000CE45CE45CE45CE45CE45CE45CE45CE4568
:10010000CE45CE45CE45CE45CE45CE45CE45CE4557
:10011000CE454B3F903F6C428542B542CC42CE45E6
:10012000CE45CE45CE45CE45CE45CE45CE45CE4537
:10013000CE45C03F1840D9425943D8431A441045D0
:100140001F459144A5442E4540455345CE45644541
:10015000FD3F25404D409845B3455B447644B94446
:10016000ED44CE03C103B303A30390037A036103F9
:10017000470329030803E602C2029E0276024F02E9
:10018000280203026C01B80196017501560139017C
:100190001F010601EF00DA00B5008200A5009600FD
:1001A000000043414E20310000000000000000002C
:1001B0000043414E2032000000000000000000001B
:1001C00043414E20330000000000000000000043C7
:1001D000414E2034000000000000000000004341B8
:1001E0004E20350000000000000000000043414E9A
:1001F00020360000000000000000000043414E20B7
:10020000370000000000000000000043414E20388D
:100210000000000000000000000043414E203900B3
:1002200000000000000000000043414E203130007B
:10023000000000000000000043414E20313100006A
:100240000000000000000043414E20313200000059
:1002500000000000000043414E2031330000000048
:10026000000000000043414E203134000000000037
:100270000000000043414E20313500000000000026
:1002800000000043414E2031360000000000000015
:10029000000043414E203137000000000000000004
:1002A0000043414E203138000000000000000000F3
:1002B00043414E203139000000000000000000439F
:1002C000414E203230000000000000000000434199
:1002D0004E20323100000000000000000043414E7B
:1002E00020323200000000000000000043414E2098
:1002F000323300000000000000000043414E203275
:100300003400000000000000000043414E20323560
:1003100000000000000000000043414E2032360083
:10032000000000000000000043414E203237000072
:100330000000000000000043414E20323800000061
:1003400000000000000043414E2032390000000050
:10035000000000000043414E203330000000000048
:100360000000000043414E20333100000000000037
:1003700000000043414E2033320000000000000026
:100380000000466C6173682031000000000000002E
:1003900000466C617368203200000000000000001D
:1003A000466C6173682033000000000000000046C6
:1003B0006C61736820340000000000000000466C8F
:1003C00061736820350000000000000000535749A9
:1003D00054434820310000000000000053574954A6
:1003E00043482032000000000000005357495443A6
:1003F0004820330000000000000053574954434890
:1004000020340000000000000053574954434820A6
:10041000350000000000000053574954434820367F
:1004200000000000000000535749544348203700A3
:100430000000000000005357495443482038000092
:100440000000000000535749544348203900000081
:100450000000000053574954434820313000000049
:100460000000005357495443482031310000000038
:1004700000004348414E4E454C2031000000000032
:10048000004348414E4E454C203200000000000021
:100490004348414E4E454C203300000000000043CD
:1004A00048414E4E454C20340000000000004348B7
:1004B000414E4E454C2035000000000000434841AD
:1004C0004E4E454C20360000000000004348414E8F
:1004D0004E454C20370000000000004348414E4E7E
:1004E000454C20380000000000004348414E4E4576
:1004F0004C20390000000000004348414E4E454C5E
:1005000020313000000000004348414E4E454C2051
:10051000313100000000004348414E4E454C20312F
:100520003200000000004348414E4E454C2031331C
:1005300000000000004348414E4E454C203134003D
:10054000000000004348414E4E454C20313500002C
:100550000000004348414E4E454C2031360000001B
:1005600000004348414E4E454C203137000000000A
:10057000004348414E4E454C2031380000000000F9
:100580004348414E4E454C203139000000000043A5
:1005900048414E4E454C2032300000000000434898
:1005A000414E4E454C20323100000000004348418E
:1005B0004E4E454C20323200000000004348414E70
:1005C0004E454C20323300000000004348414E4E5F
:1005D000454C20323400000000004348414E4E4557
:1005E0004C20323500000000004348414E4E454C3F
:1005F00020323600000000004348414E4E454C205A
:10060000323700000000004348414E4E454C203236
:100610003800000000004348414E4E454C2032391E
:1006200000000000004348414E4E454C203330004E
:10063000000000004348414E4E454C20333100003D
:100640000000004348414E4E454C2033320000002C
:1006500000004348414E4E454C203333000000001B
:10066000004348414E4E454C20333400000000000A
:100670005649525455414C203100000000000056AC
:1006800049525455414C20320000000000005649A8
:10069000525455414C20330000000000005649528E
:1006A0005455414C2034000000000000564952547B
:1006B00055414C2035000000000000564952545569
:1006C000414C20360000000000005649525455416C
:1006D0004C20370000000000005649525455414C50
:1006E00020380000000000005649525455414C206B
:1006F000390000000000005649525455414C203149
:100700003000000000005649525455414C20313110
:1007100000000000005649525455414C203132002F
:10072000000000005649525455414C20313300001E
:100730000000005649525455414C2031340000000D
:1007400000005649525455414C20313500000000FC
:10075000005649525455414C2031360000000000EB
:100760005649525455414C20313700000000005684
:1007700049525455414C2031380000000000564980
:10078000525455414C203139000000000056495266
:100790005455414C203230000000000011241FBE8F
:1007A000CFEFD0E1DEBFCDBF11E0A0E0B1E0E2EBE2
:1007B000F4EB00E00BBF02C007900D92AA37B1071F
:1007C000D9F71FE0AAE7B1E001C01D92A33AB10733
:1007D000E1F70C94042D0C940000282F2770992722
:1007E0009695879596958795969587953327233087
:1007F000310529F1243031054CF421303105B9F0AF
:1008000022303105C4F4232B71F02CC02530310582
:10081000F1F025303105BCF026303105E1F027300C
:100820003105E9F01FC0A098A198A2981BC0A09A1A
:10083000A198A29817C0A098A19AA29813C0A09AB4
:10084000A19AA2980FC0A098A198A29A0BC0A09AB2
:10085000A198A29A07C0A098A19AA29A03C0A09AB0
:10086000A19AA29A806280937C0080917A00806431
:1008700080937A0080917A0084FFFCCF80917A0087
:10088000806180937A002091780080917900992787
:10089000880F991F880F991F2295269526952370FA
:1008A000820F911D0895282F277099279695879577
:1008B000969587959695879533272330310529F1AD
:1008C000243031054CF421303105B9F022303105A6
:1008D000C4F4232B71F02CC025303105F1F0253004
:1008E0003105BCF026303105E1F027303105E9F063
:1008F0001FC0A098A198A2981BC0A09AA198A298E6
:1009000017C0A098A19AA29813C0A09AA19AA298E1
:100910000FC0A098A198A29A0BC0A09AA198A29AE1
:1009200007C0A098A19AA29A03C0A09AA19AA29ADD
:10093000806280937C0080917A00806480937A004A
:1009400080917A0084FFFCCF80917A00806180934F
:100950007A00809179009927089540E050E0FC01E9
:100960000296259134916217730760F44B5F5F4FD5
:10097000FC010296259134916217730718F44639E9
:100980005105A4F3CA010895FC0180910001813052
:10099000B1F410920001F0938301E0938201F0938F
:1009A0008101E0938001F0937F01E0937E01F09359
:1009B0007D01E0937C01F0937B01E0937A016091EB
:1009C0008001709181017093830160938201409155
:1009D0007E0150917F0150938101409380012091CD
:1009E0007C0130917D0130937F0120937E018091C5
:1009F0007A0190917B0190937D0180937C01F0932B
:100A00007B01E0937A01E80FF91FE20FF31FE40F77
:100A1000F51FCF01860F971F65E070E00E94A05977
:100A2000CB01089580E10E94ED030E94C404BC0143
:100A300082E691E00E94AD049927089583E10E9427
:100A400053049FE4899FC0011124880F892F881FB8
:100A5000990B9195A82F809101018130C1F41092DA
:100A600001018A2F992790938D0180938C01909397
:100A70008B0180938A0190938901809388019093E0
:100A80008701809386019093850180938401E09192
:100A90008A01F0918B01F0938D01E0938C016091BC
:100AA00088017091890170938B0160938A01409154
:100AB00086015091870150938901409388012091CC
:100AC00084013091850130938701209386018A2F1C
:100AD00099279093850180938401820F931F840F3F
:100AE000951F860F971F8E0F9F1F65E070E00E9475
:100AF000A059862F9927089580E280937C0087E88B
:100B000080937A00989A999A9A9AA098A198A29814
:100B1000089590E0892F8295807F8093ED00109258
:100B2000EE001092EF001092F0001092F10010927F
:100B3000F2001092F3001092F4001092F50010925F
:100B4000F6001092F70080E01092FA008F5F883074
:100B5000D8F39F5F9F30F0F208953091ED0090E060
:100B600020EC892F8295807F8093ED008091EF00AB
:100B7000822329F43093ED00892F992708959F5FF0
:100B80009F3078F33093ED008FEF90E008958091DF
:100B9000EE0086FF03C080E090E008958091EE00B3
:100BA00085FF03C081E090E008958091EF00807C94
:100BB00019F48FEF90E0089582E090E00895BC0171
:100BC00040E08091EF0099278F709070892B89F019
:100BD000FB01E40FF11D8091FA0080834F5F242F09
:100BE00033278091EF0099278F709070281739076D
:100BF0007CF308958AE39EE00E94552C60EE7EE02F
:100C000080E00E94922C68E97EE081E00E94922CB4
:100C100062E57EE082E00E94922C81E080938E016A
:100C200080913A0E813061F480913B0E90913C0EA0
:100C30006AE070E00E94A0597093390E6093380EFC
:100C40008091E10E813061F48091E20E9091E30E8B
:100C50006AE070E00E94A0597093350E6093340EE4
:100C60008091990E813061F480919A0E90919B0E43
:100C70006AE070E00E94A0597093370E6093360EC0
:100C80008091530E813061F48091540E9091550EF5
:100C90006AE070E00E94A0597093DF0E6093DE0E50
:100CA0000895CF93DF93CDB7DEB7CE55D0400FB6C2
:100CB000F894DEBF0FBECDBF19828CE0888F84E62A
:100CC00090E09B838A831D821C821E821F8218866D
:100CD00019861A861B8689819E01245F3F4FF90180
:100CE000E80FF11D10828F5F8C30C8F3CE010196A2
:100CF0000E94452CA895198E1A8E84E690E09C8F50
:100D00008B8F1E8E1D8E898D9E012F5F3F4FF901A7
:100D1000E80FF11D168E8F5F8232C8F3CE0149961F
:100D20000E94652CA89581E0898F1A8E84E690E058
:100D30009C8F8B8F1E8E1D8E8A8D9E012F5F3F4F45
:100D4000F901E80FF11D168E8F5F8232C8F3CE01D4
:100D500049960E94652CA89582E0898F1A8E84E6B8
:100D600090E09C8F8B8F1E8E1D8E8A8D9E012F5F33
:100D70003F4FF901E80FF11D168E8F5F8034C8F3E5
:100D8000CE0149960E94652CC25ADF4F0FB6F894E7
:100D9000DEBF0FBECDBFDF91CF9108959927883276
:100DA000910509F440C08932910594F4853291058A
:100DB00059F18632910534F483329105D9F0849744
:100DC000F1F04FC08632910521F1879739F149C082
:100DD0008B329105B9F18C32910534F48932910549
:100DE00039F18A9751F13DC08C32910581F18D978F
:100DF00099F137C080EC0E94CC399927089581EC95
:100E00000E94CC399927089582EC0E94CC39992709
:100E1000089581ED0E94CC399927089584EC0E94B1
:100E2000CC399927089585EC0E94CC3999270895EB
:100E300086EC0E94CC399927089587EC0E94CC3922
:100E40009927089583EC0E94CC399927089582ED63
:100E50000E94CC399927089583ED0E94CC399927B7
:100E6000089580E090E00895FF920F931F93CF9331
:100E7000DF93CDB7DEB765970FB6F894DEBF0FBE30
:100E8000CDBF8091380E9091390E009709F479C04A
:100E900001979093390E8093380E892B09F071C019
:100EA00080913B0E90913C0E6AE070E00E94A05948
:100EB0007093390E6093380E80913D0E90913E0EE6
:100EC000AA27BB2789839A83AB83BC8388E08D8361
:100ED00080918E018E8380913F0E0E94A82396956B
:100EE0008795969587958F838091400E0E94A823C1
:100EF000969587959695879588878091410E0E9453
:100F0000A823969587959695879589878091420E17
:100F10000E94A82396958795969587958A878091B4
:100F2000430E0E94A82396958795969587958B8763
:100F30008091440E0E94A823969587959695879553
:100F40008C8720918E018AE39EE0FC01E20FF11D67
:100F500082850E94A82396958795969587958D877B
:100F600080918E01982F9F5F90938E018091510EFA
:100F7000891718F481E080938E01CE0101960E94BA
:100F8000FE378091340E9091350E009709F4EDC034
:100F900001979093350E8093340E892B09F0E5C0AC
:100FA000CE010E960E9412238091E20E9091E30EE4
:100FB0006AE070E00E94A0597093350E6093340E81
:100FC0008091E40E9091E50EAA27BB2789839A832E
:100FD000AB83BC8388E08D83FF2400E81F2D812F25
:100FE0009927FC01E052F14F8681833230F40E9450
:100FF000CC22882371F0F02A0CC08E3230F40E948B
:10100000CE06882331F0F02A04C08E3211F4A49960
:10101000F02A06951F5F183010F3FE82FF2400E8C7
:101020001F2D812F9927FC01E052F14F86858332D5
:1010300030F40E94CC22882371F0F02A0CC08E324A
:1010400030F40E94CE06882331F0F02A04C08E329C
:1010500011F4A499F02A06951F5F183010F3FF824F
:10106000FF2400E81F2D812F9927FC01E052F14F4A
:101070008689833230F40E94CC22882371F0F02AD2
:101080000CC08E3230F40E94CE06882331F0F02A54
:1010900004C08E3211F4A499F02A06951F5F18300F
:1010A00010F3F886FF2400E81F2D812F9927FC01FB
:1010B000E052F14F868D833230F40E94CC22882397
:1010C00071F0F02A0CC08E3230F40E94CE068823D4
:1010D00031F0F02A04C08E3211F4A499F02A06955A
:1010E0001F5F183010F3F986FF248091060F8332BA
:1010F00048F40E94CC22882391F00F2EF0E8FF2EB6
:10110000F02D0DC08E3238F40E94CE06882339F0BF
:1011100080E8F82A04C08E3211F4A499F02A809154
:10112000070F833238F40E94CC22882381F080E4B8
:10113000F82A0DC08E3238F40E94CE06882339F08A
:1011400080E4F82A04C08E3211F4A499F02AFA86B9
:101150008E859F856AE070E00E94A0596B871C868F
:101160001D86CE0101960E94FE378091360E909129
:10117000370E009709F4E4C001979093370E8093DF
:10118000360E892B09F0DCC080919A0E90919B0E4F
:101190006AE070E00E94A0597093370E6093360E9B
:1011A00080919C0E90919D0EAA27BB2789839A83DC
:1011B000AB83BC8388E08D83FF2400E81F2D812F43
:1011C0009927FC01E856F14F8681833230F40E9462
:1011D000F222882371F0F02A0CC08E3230F40E9483
:1011E000CE06882331F0F02A04C08E3211F4A4997F
:1011F000F02A06951F5F183010F3FE82FF2400E8E6
:101200001F2D812F9927FC01E856F14F86858332E7
:1012100030F40E94F222882371F0F02A0CC08E3242
:1012200030F40E94CE06882331F0F02A04C08E32BA
:1012300011F4A499F02A06951F5F183010F3FF826D
:10124000FF2400E81F2D812F9927FC01E856F14F5C
:101250008689833230F40E94F222882371F0F02ACA
:101260000CC08E3230F40E94CE06882331F0F02A72
:1012700004C08E3211F4A499F02A06951F5F18302D
:1012800010F3F886FF2400E81F2D812F9927FC0119
:10129000E856F14F868D833230F40E94F222882383
:1012A00071F0F02A0CC08E3230F40E94CE068823F2
:1012B00031F0F02A04C08E3211F4A499F02A069578
:1012C0001F5F183010F3F986FF248091BE0E833221
:1012D00048F40E94F222882391F00F2EF0E8FF2EAE
:1012E000F02D0DC08E3238F40E94CE06882339F0DE
:1012F00080E8F82A04C08E3211F4A499F02A809173
:10130000BF0E833238F40E94F222882381F080E4F9
:10131000F82A0DC08E3238F40E94CE06882339F0A8
:1013200080E4F82A04C08E3211F4A499F02AFA86D7
:1013300088898B871C861D86CE0101960E94FE3708
:101340008091DE0E9091DF0E009709F434C1019771
:101350009093DF0E8093DE0E892B09F02CC18091D3
:10136000540E9091550E6AE070E00E94A05970935F
:10137000DF0E6093DE0E8091560E9091570EAA27D5
:10138000BB2789839A83AB83BC8388E08D83FF244A
:1013900000E81F2D812F9927FC01EE5AF14F86811D
:1013A000833230F40E94CC22882371F0F02A0CC0E2
:1013B0008E3230F40E94CE06882331F0F02A04C029
:1013C0008E3211F4A499F02A06951F5F183010F39D
:1013D000FE82FF2400E81F2D812F9927FC01EE5A81
:1013E000F14F8685833230F40E94CC22882371F03D
:1013F000F02A0CC08E3230F40E94CE06882331F0E1
:10140000F02A04C08E3211F4A499F02A06951F5FC9
:10141000183010F3FF82FF2400E81F2D812F992739
:10142000FC01EE5AF14F8689833230F40E94CC22BF
:10143000882371F0F02A0CC08E3230F40E94CE0660
:10144000882331F0F02A04C08E3211F4A499F02AD6
:1014500006951F5F183010F3F886FF2400E81F2D53
:10146000812F9927FC01EE5AF14F868D833230F49B
:101470000E94CC22882371F0F02A0CC08E3230F406
:101480000E94CE06882331F0F02A04C08E3211F477
:10149000A499F02A06951F5F183010F3F986FF24EF
:1014A00000E81F2D812F9927FC01EE5AF14F86A1EC
:1014B000833230F40E94F222882371F0F02A0CC0AB
:1014C0008E3230F40E94CE06882331F0F02A04C018
:1014D0008E3211F4A499F02A06951F5F183010F38C
:1014E000FA86FF2400E81F2D812F9927FC01EE5A70
:1014F000F14F86A5833230F40E94F222882371F0E6
:10150000F02A0CC08E3230F40E94CE06882331F0CF
:10151000F02A04C08E3211F4A499F02A06951F5FB8
:10152000183010F3FB86FF2400E81F2D812F992728
:10153000FC01EE5AF14F86A9833230F40E94F22268
:10154000882371F0F02A0CC08E3230F40E94CE064F
:10155000882331F0F02A04C08E3211F4A499F02AC5
:1015600006951F5F183010F3FC86FF2400E81F2D3E
:10157000812F9927FC01E057F14F8081833230F4AD
:101580000E94F222882371F0F02A0CC08E3230F4CF
:101590000E94CE06882331F0F02A04C08E3211F466
:1015A000A499F02A06951F5F183010F3FD86CE012E
:1015B00001960E94FE3765960FB6F894DEBF0FBE07
:1015C000CDBFDF91CF911F910F91FF900895809132
:1015D000260F9091270F885E934031F084EF91E0C1
:1015E0009093270F8093260F8FE090E09093290F20
:1015F0008093280F89E999E090932B0F80932A0F0D
:1016000010922C0F10922D0F10922E0FE6E2FFE099
:10161000A0E7B0E089E090E021E08030920719F483
:101620000E94545A0895182E0E94545A08958F9279
:101630009F92BF92CF92DF92EF92FF920F931F93F0
:10164000CF93DF93CDB7DEB7EC970FB6F894DEBF3C
:101650000FBECDBFBB240F2EF3E18F2E9924F02DAA
:10166000BE016F5F7F4F8B2D0E947B2A8B2D9927A8
:10167000889D9001899D300D989D300D1124F901B0
:10168000E157FE4F9981492F41708081887F967084
:10169000842B892B80830F2EFFE8CF2EF1E0DF2EE5
:1016A000F02DC20ED31E8A819B81F6019283818325
:1016B0008C819D81948383832E813F813683258312
:1016C00088859985908787839A8591878B8582877E
:1016D0008C8583878D8584878E8585878F85868792
:1016E0008F8D878788A1808B89A1818B8AA1828B2E
:1016F000933090F5C901AA2797FDA095BA2FBC0198
:10170000CD010E94B856DC01CB0128A539A54AA518
:101710005BA5BC01CD010E94D2557B018C018CA53B
:10172000992787FD9095A92FB92FBC01CD010E9463
:10173000B856DC01CB019C01AD01C801B7010E9484
:101740009D55DC01CB01BC01CD010E941E54DC0182
:10175000CB01F601968385838B2D9927889D900177
:10176000899D300D989D300D11240F2EFFE8CF2E4E
:10177000F1E0DF2EF02DC20ED31EF60182858330FC
:1017800098F588859985AA2797FDA095BA2FBC0161
:10179000CD010E94B856DC01CB0128A539A54AA588
:1017A0005BA5BC01CD010E94D2557B018C018CA5AB
:1017B000992787FD9095A92FB92FBC01CD010E94D3
:1017C000B856DC01CB019C01AD01C801B7010E94F4
:1017D0009D55DC01CB01BC01CD010E941E54DC01F2
:1017E000CB01F601908787832B2D3327289DC001DD
:1017F000299D900D389D900D1124FC01E157FE4F5D
:10180000808186958370813029F4F901E151FC4F84
:10181000808306C08B2D9927FC01E151FC4F10827B
:101820008B2D9927880F991FFC01E25EFB4F1182D7
:101830001082B394FFE1FB1508F012CFFE01BD96B4
:10184000A0E0B9E080E190E021E08030920719F457
:101850000E94435A03C0182E0E94435A8DA58093BC
:101860001C048EA580931D041092100410920F0486
:10187000EC960FB6F894DEBF0FBECDBFDF91CF91CF
:101880001F910F91FF90EF90DF90CF90BF909F90AE
:101890008F9008951F93CF93DF93CDB7DEB7EC976A
:1018A0000FB6F894DEBF0FBECDBF10E0A8958981BA
:1018B000887F89831B821A821D821C821F821E825E
:1018C000198618861A861B861C8681E08D871E86DF
:1018D0008F871F8E18A219A21AA280E090E0A0E8BC
:1018E000BFE388A799A7AAA7BBA71CA685E0FE010E
:1018F000B39611928A95E9F78FE0FE017096DF01A9
:10190000282F1D922A95E9F7189FC00111248E55A2
:101910009E4FBC01CF010E944359BE016F5F7F4FB4
:10192000812F0E94432A1F5F103208F4BFCFFE01AF
:10193000BD9680E1DF011D928A95E9F7A0E0B9E04C
:1019400080E190E021E08030920719F40E94545A1F
:1019500003C0182E0E94545AEC960FB6F894DEBFBE
:101960000FBECDBFDF91CF911F91089580930F04DB
:1019700008950F93CF93DF93CDB7DEB721970FB6BE
:10198000F894DEBF0FBECDBF89838150803270F0E6
:1019900000E021E0AE014F5F5F4F68E071E082E060
:1019A00091E00E94462680E090E007C08981992757
:1019B000FC01E251FC4F8081992721960FB6F894E3
:1019C000DEBF0FBECDBFDF91CF910F910895CF93B2
:1019D000DF9380911C04882381F080911D040E9474
:1019E000CC39882351F4482F8FEE93E0FC01E40FAB
:1019F000F11D10824F5F4032C8F340E06EE174E0A9
:101A0000A3E1B0E0CFEED3E051E0242F3327C901AA
:101A1000820F931FFC01E60FF71F808191810097D1
:101A200009F1019791838083892BE1F42A9FC001FA
:101A30002B9F900D3A9F900D1124FC01E157FE4F12
:101A400080818695837099278130910539F00297BE
:101A500049F0F901EC0FFD1F108204C0FE01E40FF4
:101A6000F11D50834F5F403280F2DF91CF91089596
:101A700080910F04882399F080911004882379F0D5
:101A800080E194E0AC014C5F5F4F60911304809162
:101A90001104909112040E941446109210040895AB
:101AA0008F929F92AF92BF92CF92DF92EF92FF926E
:101AB0000F931F93CF93DF938C01EE24FF2499247F
:101AC00080911C04882339F080911D040E94CC3938
:101AD000882309F42BC280912A0F90912B0F9C012F
:101AE00044275527F80180819181A281B381821713
:101AF0009307A407B50799F480912C0FE80FF11D07
:101B0000858190912D0F8923891749F40E94AD4753
:101B10000E945A1A1092380F82E28093120160E0FC
:101B200070910F040F2EFFEEAF2EF3E0BF2EF02DBD
:101B300088248394C090280FD090290F83E1689F58
:101B4000C0011124EC01C157DE4F89819A81AA2777
:101B500097FDA095BA2FF8012081318142815381F0
:101B600082179307A407B50759F08B819C81AA2798
:101B700097FDA095BA2F82179307A407B507C1F464
:101B8000462F5527CA01840F951FFC01E25EFB4FCB
:101B9000D182C082872F733048F099279C012F7320
:101BA0003070CA0103962817390711F499249394C9
:101BB0008F85882349F08889F801E80FF11D9989FC
:101BC0008581981709F05FC129813A812115310576
:101BD00009F459C1442737FD4095542FF8018081FD
:101BE0009181A281B381281739074A075B0709F061
:101BF0009CC091E08B85882379F0E80FF11D8481EA
:101C0000E82EFF24FE2CEE248C85F801E80FF11D50
:101C10008481E80EF11C14C08C85882381F0F801C2
:101C2000E80FF11D8481E82EFF248A89813041F478
:101C3000EE2034F420E03FEFE22AF32A01C090E0E6
:101C4000992309F472C08985992782309105B9F1E9
:101C5000833091052CF4009779F00197C1F065C0AD
:101C60008430910509F44DC0843091050CF43EC0D8
:101C7000059709F451C059C08D819E818E159F052D
:101C800009F053C0F501E60FF11D80824EC02A898C
:101C9000213059F48D819E818E159F050CF045C031
:101CA000F501E60FF11D208340C08D819E818E15C8
:101CB0009F05D8F5F501E60FF11D808236C02A890F
:101CC000213051F48D819E81E816F90674F5F501F5
:101CD000E60FF11D208329C08D819E81E816F9064B
:101CE00020F5F501E60FF11D80821FC08D819E81D8
:101CF0008E219F21892BC9F0F501E60FF11D80820D
:101D000014C08D819E818E219F21892B71F4F50154
:101D1000E60FF11D808209C08D819E818E159F0581
:101D200021F0F501E60FF11D80828B819C819C01E1
:101D3000442737FD4095542FF80180819181A2817D
:101D4000B381281739074A075B0709F09CC091E067
:101D50008D85882379F0E80FF11D8481E82EFF241A
:101D6000FE2CEE248E85F801E80FF11D8481E80E2B
:101D7000F11C14C08E85882381F0F801E80FF11D55
:101D80008481E82EFF248A89813041F4EE2034F4E6
:101D900020E03FEFE22AF32A01C090E0992309F402
:101DA00072C08A85992782309105B9F183309105F7
:101DB0002CF4009779F00197C1F065C0843091054B
:101DC00009F44DC0843091050CF43EC0059709F428
:101DD00051C059C08F8198858E159F0509F053C059
:101DE000F501E60FF11D10824EC08A89813059F449
:101DF0008F8198858E159F050CF045C0F501E60F83
:101E0000F11D108240C08F8198858E159F05D8F5F1
:101E1000F501E60FF11D108236C08A89813051F438
:101E20008F819885E816F90674F5F501E60FF11D26
:101E3000108229C08F819885E816F90620F5F501F2
:101E4000E60FF11D10821FC08F8198858E219F2182
:101E5000892BC9F0F501E60FF11D108214C08F81A6
:101E600098858E219F21892B71F4F501E60FF11DD4
:101E7000108209C08F8198858E159F0521F0F5018C
:101E8000E60FF11D10826F5F603208F457CE80912B
:101E90000F04882309F44AC0992019F4823009F00C
:101EA00045C080911004823009F440C08091110433
:101EB000909112049C0144275527F801808191815B
:101EC000A281B381281739074A075B0799F49091DB
:101ED00013048481981771F4892F992798012B5F37
:101EE0003F4FAC01B90180E194E004960E944A5949
:101EF000892BC9F082E080931004F801248120939B
:101F00001304808191819093120480931104822F95
:101F1000992798012B5F3F4FAC01B90184E194E010
:101F20000E94575903C081E080931004DF91CF9144
:101F30001F910F91FF90EF90DF90CF90BF90AF90E7
:101F40009F908F9008950E9489058091D8008260AB
:101F50008093D8000895CF93DF93EC01898183307B
:101F600089F48985882309F403C188818295807F5B
:101F70008093ED008091EF008F738093EF001882C3
:101F80001986F6C00E94AD05982F81E089879F3F92
:101F900009F4EBC09883892F8295807F8093ED00B0
:101FA0001092EE001092EF001092F7001092F600DF
:101FB0001092F5001092F4001092F0008981992798
:101FC0008130910509F46BC0823091051CF4892B96
:101FD00029F0C9C0029709F4BBC0C5C08A8581FF3A
:101FE00030C08D81982F990F990F990F8C81829510
:101FF00086958770890F8093F3008C81982F990FB5
:10200000990F990F8B81829586958770890F8093A0
:10201000F2008B81982F990F990F990F8A818295E1
:1020200086958770890F8093F1008A81880F880FC9
:10203000880F8093F0008091EF0080618093EF0023
:1020400012C08B81982F9295990F907E8A818695E8
:1020500086958695890F8093F3008A818295880FF3
:10206000807E8093F20020E08E81181660F48F81CC
:102070009885FC01E20FF11D80818093FA002F5FAB
:102080008E812817A0F39091EF008E81892B809389
:10209000EF008091EF0080648093EF0069C08A8533
:1020A00081FF35C08D81982F990F990F990F8C81E1
:1020B000829586958770890F8093F3008C81982F85
:1020C000990F990F990F8B81829586958770890F4B
:1020D0008093F2008B81982F990F990F990F8A8125
:1020E000829586958770890F8093F1008A81880F89
:1020F000880F880F8093F0008091EF0080618093BB
:10210000EF008091F00084608093F00015C08B8117
:10211000982F9295990F907E8A81869586958695BF
:10212000890F8093F3008A818295880F807E809347
:10213000F20084E08093F0009091EF008E81892B73
:102140008093EF008091EF0080648093EF0010C0D7
:102150008091EF008F738093EF008091EF00806893
:102160008093EF0005C0198603C08FEF90E002C096
:1021700080E090E0DF91CF910895CF93DF93EC0161
:102180008985882319F482E090E082C08881829555
:10219000807F8093ED000E94C705813009F06CC0FC
:1021A00019868091EF008F708E838F8198850E94B1
:1021B000DF058091F0009927847090709595879540
:1021C00095958795982F91708A85282F2E7F292B9A
:1021D0002A878091EF0084FF31C0822F82608A8736
:1021E0008091F3008695869586958D838091F20087
:1021F000982F9695969596958091F3008295880FE5
:10220000807E890F8C838091F100982F969596950A
:1022100096958091F2008295880F807E890F8B833E
:102220008091F000982F9695969596958091F10063
:102230008295880F807E890F8A8316C08A858D7F5C
:102240008A878091F3008295869587708B83809131
:10225000F200982F9295969597708091F300880FD1
:10226000880F880F890F8A838091EF008F73809386
:10227000EF0080E090E00CC0882349F489878091CA
:10228000EF008F738093EF0080E090E001C099270A
:10229000DF91CF910895982F8F3F19F481E090E05E
:1022A0000895805C843128F4892F0E94CC399927C5
:1022B0000895892F8150803228F4892F0E94B90C0B
:1022C00099270895892F8152843128F4892F0E94FB
:1022D000E74B9927089580E090E008958091310FB1
:1022E0000E944B11882321F085E080935B0A41C056
:1022F0008091360F0E944B11882341F08091370F57
:1023000080935D0A83E080935B0A33C08091300F35
:102310000E944B11882321F084E080935B0A29C03E
:102320008091320F0E944B11882341F080915B0A0B
:10233000873021F086E080935B0A1BC080915B0AA6
:10234000853021F482E080935B0A13C080915B0AA0
:10235000833041F480915D0A882321F481E08093E9
:102360005B0A07C080915B0A843019F481E0809396
:102370005B0A80915B0A8150823058F48091330F60
:102380000E944B119091340F981719F410925B0A28
:1023900013C080915B0A863079F48091330F0E94DC
:1023A0004B119091340F981739F487E080935B0AB2
:1023B0008091350F80935C0A86ED99E00E949E24FF
:1023C0000E94C61208951F93CF93DF930E94731A41
:1023D0000E94C5190E94DF1B10E087E2189FC00110
:1023E0001124EC01CB59DB4F8C899D89009719F0A2
:1023F00001979D8B8C8B8D859E85009761F0019751
:102400009E878D8799859F3F31F085E0989FC00119
:1024100011249B878A872A853B852115310561F028
:1024200089858F3F49F0C90101979B878A87892B4E
:1024300019F48F8580628F878B8D9C8D009779F042
:1024400001979C8F8B8F892B51F48F8586FD04C05B
:10245000812F8F5F0E9424298F8580648F878F81D1
:10246000882311F081508F831F5F123208F4B5CF9B
:10247000DF91CF911F91089580915B0A8730A1F47D
:1024800080915C0A882321F0815080935C0A0CC003
:102490008091320F0E944B11882321F086E08093B7
:1024A0005B0A02C010925B0A80915D0A882319F0D2
:1024B000815080935D0AA49B23C02091580A2F3736
:1024C00010F4220F01C02FEF80912E0F8A30D0F030
:1024D00090912F0F981710F0921730F480912F0FD2
:1024E0008F5F80932F0F0EC08091380F882351F497
:1024F0008F5F8093380F0E94AD470E945A1A02C026
:1025000010922F0F9091CD098091DD099817E0F47A
:1025100020E04DED59E067E270E0FA01E20FF11DB5
:102520008281823268F49927869FF001879FF00D9F
:10253000969FF00D1124E759FB4F808181608083C5
:102540002F5F2C3050F308959091CD098091DE09D2
:102550008917D8F420E04DED59E067E270E0FA0108
:10256000E20FF11D8281823268F49927869FF00183
:10257000879FF00D969FF00D1124E759FB4F808146
:102580008E7F80832F5F2C3050F30895CF92DF929F
:10259000EF92FF920F931F93CF93DF9380915F048D
:1025A000882309F004C1F82E0F2EFAE0EF2EF02D4B
:1025B0008EE0F89EC0011124EC01CE5ED54F00E004
:1025C0008A818F3F11F401E01DC09A81892F805CC0
:1025D000843128F4892F0E94CC39082F13C09A81A6
:1025E000892F8150803228F4892F0E94B90C082F3E
:1025F00009C09A81892F8152843120F4892F0E9449
:10260000E74B082F8981992781309105C9F18230E4
:1026100091051CF4892B29F0C5C0029709F4BFC0AD
:10262000C1C0013009F0BEC08F818E9DC001112450
:102630009C838B8389858E9DC00111249E838D830D
:1026400088818460888310E027E230E0FE01E10F9A
:10265000F11D82858F3F71F09927829FA001839F92
:10266000500D929F500D1124FA01E759FB4F8081C4
:10267000846080831F5F143048F381E0898392C0B7
:102680008B819C81009709F48DC001979C838B837B
:10269000892B81F5288122FF17C08F818E9DC00173
:1026A00011249C838B83822F8B7F888310E0FE0113
:1026B000E10FF11D82858F3F19F060E00E94E01369
:1026C0001F5F1430A0F316C088858E9DC0011124B1
:1026D0009C838B8388818460888310E0FE01E10FF6
:1026E000F11D82858F3F19F061E00E94E0131F5FAA
:1026F0001430A0F38881282F227081FD28C08D819D
:102700009E81009709F44EC001979E838D83892B8B
:1027100009F048C082E08983122F27E230E0FE01F1
:10272000E10FF11D82858F3F71F09927829FA001F3
:10273000839F500D929F500D1124FA01E759FB4FD2
:1027400080818B7F80831F5F143048F32BC0002370
:1027500049F5102F0F2EF7E2CF2EDD24F02DFE01CC
:10276000E10FF11D22852F3F99F0822F99278C9D33
:10277000A0018D9D500D9C9D500D1124FA01E7592B
:10278000FB4F80818B7F808361E0822F0E94E0136A
:102790001C821B821F5F143010F3198203C00023B8
:1027A00009F40983F39454E05F1508F001CFDF9139
:1027B000CF911F910F91FF90EF90DF90CF900895F0
:1027C000DF92EF92FF920F931F93CF93DF93CDB7DA
:1027D000DEB721970FB6F894DEBF0FBECDBF898359
:1027E000162FDD24833260F00D2D21E0AE014F5F06
:1027F0005F4F64E372E083E191E00E9446264EC0A1
:10280000998187E2989F7001112485E694E0E80E93
:10281000F91EF701868D9927807F9070803A910587
:1028200029F40F2EF1E4DF2EF02D18C0F701868D6C
:102830009927807F9070803B910529F40F2EF2E458
:10284000DF2EF02D0BC000E021E0AE014F5F5F4FA7
:1028500060E472E083E191E00E944626112379F45E
:1028600083E0F701878380EF818387858F7B87876C
:10287000868D42A16D2D8F700E9452320FC0113093
:1028800069F4F70117828FE08183878586798787CE
:10289000868D42A16D2D8F700E949D3221960FB6BC
:1028A000F894DEBF0FBECDBFDF91CF911F910F9186
:1028B000FF90EF90DF90089520E04BEE59E067E243
:1028C00070E08170382F330FFA01E20FF11D818122
:1028D000823270F49927869FF001879FF00D969FB2
:1028E000F00D1124E759FB4F80818D7F832B80836E
:1028F0002F5F2E3048F3089520E04BEE59E067E259
:1029000070E08170382F330FFA01E20FF11D8189D9
:10291000823270F49927869FF001879FF00D969F71
:10292000F00D1124E759FB4F80818D7F832B80832D
:102930002F5F2E3048F308958091610490916204D6
:1029400008958091600499270895EF92FF921F9354
:10295000CF93DF937A018093DD096093DE0910E065
:10296000C12FDD27F701EC0FFD1F80810E94392167
:10297000823220F4FE01E352F64F82831F5F1C3047
:1029800078F3DF91CF911F91FF90EF900895AF9270
:10299000BF92CF92DF92EF92FF920F931F93CF934C
:1029A000C0E00E942C230E941B240E94462486ED36
:1029B00099E00E9493241092CB091092CA09C09307
:1029C000CC09C093CE09C093CF09C093D009C0935E
:1029D000D10982E1E3E9F9E011928A95E9F745EA44
:1029E00059E028EB31E08C2F9927880F991FFC01C3
:1029F000E40FF51F31832083CF5FC231A0F3C0E025
:102A000042E15AE02EE030E08C2F9927829FB001FE
:102A1000839F700D929F700D1124FB01E40FF51F31
:102A200011821482138216821582FB01EE5EF54F2D
:102A3000808184608083CF5FC53030F30E94D32CC7
:102A4000803221F487E68093110103C08EE68093E3
:102A50001101A5E6B4E021E02093650448EC50E0C4
:102A6000509378044093770432EA3093830462EB06
:102A700060938404109287049FEF909385043093B1
:102A8000860415E01093880483E0809389040F2E58
:102A9000F7E2CF2EDD24F02DCA0EDB1E20938C042E
:102AA000FD0152AF41AFF601368F678F22A390A38D
:102AB0000F2EF7EAFF2EF02DF1A213A38FE084A3CF
:102AC000FD01E25BFF4F2093B304538B428B0F2E2B
:102AD000F3EAEF2EF02DE68E83EB878F22A390A3EF
:102AE00091A393A389E084A3FD01EB58FF4F2093AA
:102AF000DA04538B428BF68E0F2EF7EBCF2EF02D90
:102B0000C78E22A390A391A393A38BE084A3FD017E
:102B1000E456FF4F20930105538B428B0F2EF1EAB1
:102B2000DF2EF02DD68E81EB878F22A390A391A369
:102B300093A38EE084A3FD01ED53FF4F209328055E
:102B4000538B428B35EA368F05EB078F22A390A378
:102B500091A393A38DE084A3C6E0FD01E651FF4F4E
:102B600020934F05538B428B60EA668F70EB778F13
:102B700012A290A331A313A3C4A3FD01EF5EFE4FE5
:102B800020937605538B428B368F078F12A290A32A
:102B900091A393A384E084A3FD01E85CFE4F2093FE
:102BA0009D05538B428B668F778F22A390A361A3E1
:102BB00013A38AE084A3FD01E15AFE4F2093C405CC
:102BC000538B428B768F34EB378F12A390A391A354
:102BD00093A382E184A3FD01EA57FE4F2093EB0506
:102BE000538B428B64EA668F378F22A390A3E1A2B6
:102BF00013A388E084A3FD01E355FE4F2093120642
:102C0000538B428B36EA368F86EB878F12A290A3C6
:102C100061A313A324A3CCE0FD01EC52FE4F20934B
:102C20003906538B428B368F878F22A390A3D1A274
:102C300013A3C4A3FD01E550FE4F20936006538B00
:102C4000428BF68EC78E12A290A391A393A3CC249D
:102C50006894C1F8C4A29D01FD01EE5DFD4F71E0D5
:102C600070938706538B428BBD2CD68E0F2EF1EBC3
:102C7000EF2EF02DE78E12A290A391A393A387E0ED
:102C800084A3FD01E75BFD4F7093AE06538B428B2F
:102C9000E68EF02E078F612F12A390A391A393A32A
:102CA00081E184A3FD01E059FD4F7093D506538B5C
:102CB000428B14EA168FB4EBB78F12A290A386EA68
:102CC00081A363A364A3F901E956FD4F7093FC0649
:102CD000538B428B0F2EF3EAAF2EF02DA68E03EB13
:102CE000078F12A290A391A393A314A2F901E25417
:102CF000FD4F70E4709323074FEF5FEF538B428BD0
:102D0000A7EAA68FB78F63E062A380A391A393A3E2
:102D100094A3F901EB51FD4F70934A07538B428BFB
:102D2000868FF78E62A380A391A393A394A3F90146
:102D3000E45FFC4F70937107538B428BB5EAB68FFB
:102D400086EB878F62A3A0A391A393A394A3F90119
:102D5000ED5CFC4F70939807538B428B168F87EB7B
:102D6000878F62A3A0A391A393A394A3F901E65A2A
:102D7000FC4F7093BF07538B428B0F2EF0EADF2E70
:102D8000F02DD68E078F62A3B0A391A393A394A333
:102D9000F901EF57FC4F7093E607538B428BB68EC9
:102DA000A2EBA78F62A3B0A391A393A394A3F9016D
:102DB000E855FC4F70930D08538B428B82EA868F47
:102DC000E78E62A310A391A393A394A3F901E15307
:102DD000FC4F70933408538B428BA68E80EB878F09
:102DE00062A310A391A393A394A3F901EA50FC4F0B
:102DF00070935B08538B428BD68E078FC2A2F0A2D2
:102E000091A393A394A3F901E35EFB4F709382080F
:102E1000538B428BB68EA78FC2A2F0A291A393A32D
:102E2000F901E35EFB4F94A3B901F901EC5BFB4FA1
:102E3000A0E4A093A908538B428B82EA868FE78E89
:102E4000C2A224EB20A391A393A394A3FB01E55971
:102E5000FB4FA093D008538B428BA68E80EB878FBD
:102E6000C2A220A391A393A394A3FB01EE56FB4F10
:102E7000A093F708538B428B87EA868F278FC2A2D5
:102E800026EB20A391A393A394A3FB01E754FB4F4C
:102E9000A0931E09538B428B86EA868FF78EC2A2BF
:102EA00020A391A393A394A3FB01E052FB4FA09313
:102EB0004509538B428BB68F278FC2A227EB20A3E5
:102EC00091A393A394A3FB01E95FFA4FA0936C092C
:102ED000538B428B168F278FC2A220A391A393A35B
:102EE00094A3C0E047E250E02FE001E21EE130E1B0
:102EF0008C2F9927849FF001859FF00D949FF00DF2
:102F00001124CF01E60FF71F158A148A168ADC01F7
:102F1000A759BB4F8C918C7F8C931786178A21837E
:102F200016A215A216861586148613861286118699
:102F30008C918B7F8C93108E17820087168335833C
:102F40002283128E118E148E138E158ECF5FC23295
:102F500078F2CF911F910F91FF90EF90DF90CF907B
:102F6000BF90AF900895E3E9F9E082E1DF011D929F
:102F70008A95E9F7CF010E94052C20E065EA79E007
:102F800048EB51E0822F9927880F991FFC01E60F2B
:102F9000F71F518340832F5F2231A0F385EA99E028
:102FA0000E94252C0895AF92BF92CF92DF92EF92AC
:102FB000FF920F931F93CF93DF93CDB7DEB7C35725
:102FC000D0400FB6F894DEBF0FBECDBFDD240F2E6C
:102FD000F5E1EF2EFF24F02DEC0EFD1E2D2D3327F5
:102FE00087E290E0289FA001299F500D389F500D47
:102FF0001124FA01EB59FB4F82899389892F992774
:103000008D8B82898E8B86818F8B1A8E198E1B8E6B
:103010008581888F80858C8F8FE0D89EC001112498
:103020008E589B4FBC01CE014D960E9443591CA661
:103030001DA61D2D1F5F612FC7010E94232BA89580
:10304000D12E51E2511750F684E68EA788E78FA75C
:103050004CE050E06FEF70E0CE01C0960E946459E2
:10306000CE018E960E94632981EC8CAF8E01045CA8
:103070001F4F4EE050E06FEF70E0CE01CD960E9402
:103080006459FE01E55BFF4F10828AE0FE01E45BBC
:10309000FF4F80834EE050E06FEF70E0C801419633
:1030A0000E946459C8010E949129A895DD240F2E21
:1030B000F4E1CF2EF02D7E010894E11CF11C0FE00D
:1030C000D701EC2D1D92EA95E9F7D09EC00111249D
:1030D00083539C4FBC01C7010E944359188A1D2D80
:1030E0001F5FB701812F0E94BA2BD12EFAE0F11792
:1030F00038F7A895DD240F2EF5E6AF2EBB24F02D72
:10310000AC0EBD1E0F2EFFE0CF2EF02D8E01055A06
:103110001F4FEE24E394FF24FA94D501EC2D1D9269
:10312000EA95E9F7DC9CC00111248E579C4FBC0145
:10313000C8010A960E944359D8011C92F8011182D5
:103140001282E382E4828AE085838081F801E80FBD
:10315000F11DF6828F5F8430C8F3BE01655A7F4F40
:103160008D2D0E94D129D394F4E0FD15B0F6EAE04C
:10317000FAE018E0DF01212F1D922A95E9F7CF012F
:103180000E94B1290E940E24E0E3FFE0DF011D92BE
:103190001A95E9F781E08093340F8EE18093350F23
:1031A00082E38093370FA2E9BFE088E090E021E05E
:1031B0008030920719F40E94545A03C0182E0E94BE
:1031C000545ACD58DF4F0FB6F894DEBF0FBECDBFB7
:1031D000DF91CF911F910F91FF90EF90DF90CF90F3
:1031E000BF90AF9008950F931F93CF93DF93CDB708
:1031F000DEB7E2970FB6F894DEBF0FBECDBF00E09A
:10320000102F1F5F612FCE0101960E94682B202F87
:10321000332787E290E0289FA001299F500D389F17
:10322000500D1124FA01EB59FB4F89819927982FF2
:1032300088272A81820F911D938B828B8B818683B5
:10324000888580878C818583888D8487898D818717
:103250008D819E81928F818F8F81858F012F123278
:1032600078F28DED99E00E9481298BEE99E00E9421
:10327000A12983E999E00E94152C85EA99E00E9432
:10328000352C8AE09AE00E94C1290E940E2400E0B9
:10329000BE01665E7F4F802F0E940A2A202F3327AF
:1032A0008EE090E0289FA001299F500D389F500D7F
:1032B00011249A01FA01EE5EF54F8A8D582F517054
:1032C0008081482F4C7F8B8D8170982F990F842F90
:1032D000852B892B8083F901EE5EF54F8C8D8283DF
:1032E0008D8D87838E8D80878F8D8187F901E45E38
:1032F000F54F88A199A1AAA1BBA180839183A28344
:10330000B3830F5F053020F2E0E3FFE0A2E9BFE006
:1033100088E090E051E08030950719F40E94435A0C
:1033200003C0182E0E94435AE2960FB6F894DEBFEF
:103330000FBECDBFDF91CF911F910F910895CF9315
:10334000DF93EC01862F0E9439218332D8F4282F95
:10335000332787E290E0289FA001299F500D389FD6
:10336000500D1124FA01EB59FB4F8F898487888116
:103370009927982F88272981820F911D938B828B03
:103380008A818683DF91CF9108951F93CF93C0E008
:103390001C2F9091EB09892F8150803238F4892FAE
:1033A0000E94B90C8823B1F011E014C09091EB0990
:1033B000892F8152843138F4892F0E94E74B88236A
:1033C00049F011E007C08091EB090E94CC398130AF
:1033D00009F4182F9091FA09892F8150803220F436
:1033E000892F0E94B90C0EC09091FA09892F815241
:1033F000843120F4892F0E94E74B04C08091FA09A0
:103400000E94CC398E3FF1F08130B9F48091590A95
:10341000843020F48F5F8093590A09C01092590AB2
:1034200080915A0A882319F0815080935A0A80911A
:103430005A0A882359F4C1E009C08091FB0980939E
:103440005A0A04C08091FB0980935A0A113021F472
:10345000812F0E945C140CC0C13021F48C2F0E947B
:103460007C1406C080E00E945C1480E00E947C1402
:10347000CF911F910895FC0184818860848380EF3F
:103480008283878586798787178A168A848525E0CF
:10349000829FC001112496878587892B41F48185FD
:1034A0008F3F29F0829FC00111249387828783E098
:1034B000878308951F93CF93C0E017E2C19FC00197
:1034C0001124FC01EB59FB4F8785992783FD02C02E
:1034D00080FF03C0CF010E943B1ACF5FC23270F35E
:1034E000CF911F910895FF920F931F93CF93DF9376
:1034F00010E00F2EFFE0FF2EF02D82E00E944E3AEA
:1035000087E2189FC0011124EC01CB59DB4F88855D
:10351000882361F48981803F09F0EAC08C8188604A
:103520008C838F85867B8F87FA82E2C02885822FE5
:1035300081508032D0F58F85992783FD24C080FD8E
:1035400022C0822F0E94B90C882341F089818F30DC
:1035500009F0CEC0CE010E943B1ACAC08981803FCB
:1035600009F0C6C089858F3F09F4C2C08A859B8552
:10357000892B09F0BDC08C8188608C838F85867B08
:103580008F87FA82B5C088850E94B90C882309F01C
:10359000AFC08981803F09F0ABC08C8188608C838B
:1035A0008F85867B8F87FA82A3C02885822F8152E0
:1035B0008431D0F58F85992783FD24C080FD22C0FA
:1035C000822F0E94E74B882341F089818F3009F0D8
:1035D0008FC0CE010E943B1A8BC08981803F09F0C9
:1035E00087C089858F3F09F483C08A859B85892B95
:1035F00009F07EC08C8188608C838F85867B8F8765
:10360000FA8276C088850E94E74B882309F070C053
:103610008981803F09F06CC08C8188608C838F85A4
:10362000867B8F87FA8264C000E08885853371F4D9
:1036300090915B0A892F8350823020F0913011F0F5
:10364000963011F491E013C090E011C08885863364
:1036500051F480915B0A853011F0823011F491E0D1
:1036600006C090E004C088850E94CC39982F9E3F08
:10367000A9F08885803C21F49130A1F4092F12C073
:103680008D81813021F4913011F4092F0BC08D818F
:10369000803141F4992331F401E004C088858F3FE3
:1036A00009F401E0002369F089818F3009F58F85E5
:1036B000992783FD1DC080FD1BC0CE010E943B1ACF
:1036C00017C08981803F31F08F85992783FD02C023
:1036D00080FF0EC089858F3F59F08A859B85892B95
:1036E00039F48C8188608C838F85867B8F87FA8202
:1036F00089818F3079F48F85992789709070892B13
:1037000049F480911201811729F482E28093120119
:103710001092380F1F5F123208F4EFCEDF91CF9175
:103720001F910F91FF90089560935F04623019F428
:103730008FEF8093C9090895CF93DF93EC018881BF
:103740008150823218F080E090E036C088810E947B
:103750003921282F898199278F30910521F0803FC9
:103760009105A1F027C0332787E290E0289FA001B0
:10377000299F500D389F500D1124FA01EB59FB4F32
:103780008FE081838785867F878714C0332787E210
:1037900090E0289FA001299F500D389F500D1124C3
:1037A000FA01EB59FB4F80EF81838785867F8787FE
:1037B000178A168A81E090E0DF91CF9108958F9269
:1037C0009F92AF92BF92CF92DF92EF92FF920F93B0
:1037D0001F93CF93DF93CDB7DEB721970FB6F89441
:1037E000DEBF0FBECDBFBB24B9828B2CAB2C9B2C74
:1037F0001092CB091092CA09B092CE09B092D009AA
:10380000B092CF090E941E058093CD0980915F047C
:10381000882309F07AC2B9828B2D823208F0F4C471
:1038200082E00E944E3A8824998187E2989FC001E5
:1038300011240F2EF5E6CF2EF4E0DF2EF02DC80E6A
:10384000D91EF601868D9927807F9070803A910568
:1038500029F40F2EF1E4AF2EF02D18C0F601868D5D
:103860009927807F9070803B910529F40F2EF2E418
:10387000AF2EF02D0BC000E021E0AE014F5F5F4F97
:103880006EED76E083E191E00E944626F601118A12
:10389000108A248122FDBCC0808199278130910546
:1038A00009F45DC08034910509F0BFC0818199277A
:1038B0008F309105B1F1803F910509F0B6C0822F9C
:1038C000837019F4878585FF09C0F601868D42A1B2
:1038D0006A2D8F700E949D32882410C0F601858564
:1038E0009685892B59F4878580FD08C0868D42A175
:1038F0006A2D8F700E94523288248394F60184814D
:1039000083FF93C0877F848382818F3009F08DC0CD
:103910008183868D42A16A2D8F700E949D328824FA
:1039200084C0F601248123FF80C0822F877F848397
:103930008281803F09F079C0818385859685892BB6
:1039400009F073C0822F837009F06FC0868D42A189
:103950006A2D8F700E9452328824839466C0F601CB
:10396000818199278F309105C1F1803F910509F040
:103970005CC08481837019F4878585FF09C0F601D6
:10398000868D42A16A2D8F700E949D32882413C0BB
:10399000F60185859685892B71F48785992780FDA9
:1039A0000AC083FD08C0868D42A16A2D8F700E94D7
:1039B000523288248394F601848183FF36C0877F46
:1039C000848382818F3089F58183868D42A16A2D1F
:1039D0008F700E949D32882428C0F601248123FF25
:1039E00024C0822F877F84838281803FF1F481838A
:1039F00085859685892BC9F4822F8370B1F4868DD5
:103A000042A16A2D8F700E945232882483940DC087
:103A1000F601818199278F30910531F0803F910522
:103A200021F48824839401C08824F6018181803F99
:103A300009F058C084A18F3F09F454C00E94ED03DF
:103A40007C0100271127F601F6A2E5A289819927BA
:103A5000FC01ED56F64F80819927AA27BB278E15CA
:103A60009F05A007B10724F0EE24FF2487010AC0B8
:103A700089819927FC01ED56F64F8081E81AF108FB
:103A800001091109F3E0EF16F10401051105CCF06D
:103A900089819927880F991FFC01EB55F64F80818A
:103AA00091819C0144275527C801B7010E9475598F
:103AB00020EE31E040E050E00E94E95979018A01AE
:103AC00003C0EE24FF248701F601F18AE08A809189
:103AD000CA099091CB098E0D9F1D9093CB098093BD
:103AE000CA0903C0F601118A108A882039F4F60148
:103AF000838D948D892B11F0148E138EF60187859A
:103B00009927AC014870507083FD6DC020893189C0
:103B10008289938982179307D8F5838D948D892B99
:103B200011F0548F438FF6018689813031F58489F5
:103B30009589892B09F057C0878588608787809190
:103B4000CE098F5F8093CE098081813071F4868D9C
:103B500042A16A2D8F700E949D32882489818093B2
:103B60001201F60186818093580A8981F6016089E5
:103B700071898F5F0E94B92836C081E0F601868B7B
:103B8000968185E0989FC0011124958B848B2BC072
:103B9000F601168A218D328D2115310521F18820FB
:103BA000A1F0808991898217930778F4838D948D91
:103BB000892BC9F4878586FD16C0958D85E0989F71
:103BC000C0011124948F838F0EC0F601838D948DD4
:103BD000892B49F020893189818D928D8217930735
:103BE00010F4148E138EF601878D9927807F9070C4
:103BF000803A910529F40F2EF1E49F2EF02D18C084
:103C0000F601878D9927807F9070803B910529F47C
:103C10000F2EF2E49F2EF02D0BC000E021E0AE014C
:103C20004F5F5F4F66EF77E083E191E00E944626A9
:103C3000F601878D42A1692D8F700E942033282FB5
:103C4000F6018181803F09F043C08785992783FD74
:103C50003FC080FD3DC09091CD0980911101891731
:103C6000B8F5F1E08F1691F5222381F5F6018781F1
:103C7000882371F58485882359F5808D8F3F11F055
:103C80008F5F808FF601808D863010F187898F5F7E
:103C9000878B843158F4868D42A16A2D8F700E94E3
:103CA0009D32F601108E83E0878312C0F601868D67
:103CB00042A16A2D8F700E949D32F6018785816036
:103CC000878789818F5F0E94F12802C0F601108EDC
:103CD000F601878580FF05C08091D0098F5F8093B2
:103CE000D009F601878583FF05C08091CE098F5FDB
:103CF0008093CE09F60187858111B39489818F5F06
:103D00008983823208F48CCD7FC280915F04813038
:103D100009F0ADC119828981482F823208F074C23E
:103D2000242F332787E290E0289FB001299F700D50
:103D3000389F700D1124FB01EB59FB4F87858F7D58
:103D4000878787E2489FC00111240F2EF5E6CF2E0A
:103D5000F4E0DF2EF02DC80ED91EF601868D9927CE
:103D6000807F9070803A910529F40F2EF1E4AF2EF8
:103D7000F02D0CC0F601868D9927807F9070803BD6
:103D8000910521F40F2EF2E4AF2EF02DF60184817F
:103D900082FD4FC0808199278130910569F180347F
:103DA000910509F046C0818199278F30910561F016
:103DB000803F9105F1F5868D42A16A2D8F700E949A
:103DC00052328824839435C08981282F332787E293
:103DD00090E0289FA001299F500D389F500D11247D
:103DE000FA01EB59FB4F868DF60142A16A2D8F70C7
:103DF0000E949D3288241DC0F601818199278F3051
:103E0000910561F0803F9105A1F4868D42A16A2D54
:103E10008F700E945232882483940BC0F601868DE5
:103E200042A16A2D8F700E949D328FE0F60181833E
:103E30008824F6018181803F09F057C084A18F3F1B
:103E400009F453C00E94ED037C0100271127F601FD
:103E5000F6A2E5A289819927FC01ED56F64F8081F3
:103E60009927AA27BB278E159F05A007B10724F025
:103E7000EE24FF2487010AC089819927FC01ED56B1
:103E8000F64F8081E81AF10801091109F3E0EF16F5
:103E9000F10401051105CCF089819927880F991F3C
:103EA000FC01EB55F64F808191819C0144275527F9
:103EB000C801B7010E94755920EE31E040E050E0A2
:103EC0000E94E95979018A0103C0EE24FF24870189
:103ED000F601F18AE08A8091CA099091CB098E0D92
:103EE0009F1D9093CB098093CA09F60120893189DF
:103EF000828993898217930780F58689813011F52D
:103F000084899589892B69F5878588608787809161
:103F1000CE098F5F8093CE098081813059F4868DE0
:103F200042A16A2D8F700E949D3288248FE0F60195
:103F3000818382838981F601608971898F5F0E9404
:103F4000B9280FC081E0F601868B968185E0989FA5
:103F5000C0011124958B848B04C0F601168A158A42
:103F6000148AF601878D9927807F9070803A910599
:103F700029F40F2EF1E49F2EF02D0CC0F601878D51
:103F80009927807F9070803B910521F40F2EF2E4F9
:103F90009F2EF02DF601878D42A1692D8F700E9412
:103FA0002033282FF6018785992783FD42C080FDA5
:103FB00040C09091CD09809111018917D0F5F1E0B1
:103FC0008F16A9F5222399F5F6018781882389F5B3
:103FD0008485882371F58181803F59F5808D8F3FDD
:103FE00011F08F5F808FF601808D863010F1878908
:103FF0008F5F878B843158F4868D42A16A2D8F7034
:104000000E949D32F601108E83E0878312C0F60174
:10401000868D42A16A2D8F700E949D32F6018785A0
:104020008160878789818F5F0E94F12802C0F60135
:10403000108EF601878580FF05C08091D0098F5FC3
:104040008093D009F601878583FF05C08091CE0952
:104050008F5F8093CE09F60187858111B3948981A2
:104060008F5F8983482F823208F45ACECDC0809169
:104070005F04823009F0C8C019828981982F82328A
:1040800008F0C2C087E2989FC00111240F2EF5E608
:10409000CF2EF4E0DF2EF02DC80ED91EF601868D4E
:1040A0009927807F9070803A910529F40F2EF1E4D2
:1040B000AF2EF02D0CC0F601868D9927807F907071
:1040C000803B910521F40F2EF2E4AF2EF02D4091AC
:1040D000C9094423D1F0898199279C012F5F3F4F63
:1040E000842F99272817390741F4F601868D42A1BC
:1040F0006A2D8F700E9452320FC0F601868D42A148
:104100006A2D8F700E949D3207C0F601868D42A1F4
:104110006A2D8F700E945232F60184A18F3F09F4FC
:104120006CC00E94ED037C0100271127F601F6A266
:10413000E5A280915E0480FF1CC089819927FC0163
:10414000ED56F64F80819927AA27BB278E159F052C
:10415000A007B10724F0EE24FF2487010AC089815B
:104160009927FC01ED56F64F8081E81AF108010904
:104170001109F3E0EF16F1040105110574F18091C6
:104180005E0481FF19C089819927880F991FFC015E
:10419000EB55F64F808191819C0144275527C8013A
:1041A000B7010E94755920EE31E040E050E00E94D6
:1041B000E95979018A0114C0C801B70128EB31E03F
:1041C00040E050E00E94755920EE31E040E050E0C0
:1041D0000E94E95979018A0103C0EE24FF24870176
:1041E000F601F18AE08A8091CA099091CB098E0D7F
:1041F0009F1D9093CB098093CA0989818F5F898322
:10420000982F823208F43ECFBB2031F4B092CF0910
:10421000B092D009B092D1090E941205982F8093D4
:10422000CC0980916004891710F490936004209168
:10423000CA093091CB098091610490916204821780
:10424000930720F4309362042093610421960FB603
:10425000F894DEBF0FBECDBFDF91CF911F910F91BC
:10426000FF90EF90DF90CF90BF90AF909F908F9096
:104270000895815099270895CF93DF93EC01862FFD
:104280000E943921833278F4282F332787E290E087
:10429000289FA001299F500D389F500D1124FA012D
:1042A000EB59FB4FC683DF91CF910895EF92FF92B8
:1042B0001F93CF937C01C0E080EC0E94CC39811128
:1042C000C1E081EC0E94CC398111C26082EC0E9475
:1042D000CC398111C46081ED0E94CC398111C86054
:1042E00084EC0E94CC398111C06185EC0E94CC39EC
:1042F0008111C06286EC0E94CC398111C06487ECC8
:104300000E94CC398111C06810E083EC0E94CC3946
:10431000811111E082ED0E94CC398111126083ED90
:104320000E94CC3981111460F701C0831183C0E071
:1043300081E00E94B90C8111C1E082E00E94B90CB9
:104340008111C26083E00E94B90C8111C46084E0D5
:104350000E94B90C8111C86085E00E94B90C8111DE
:10436000C06186E00E94B90C8111C06287E00E94A2
:10437000B90C8111C06488E00E94B90C8111C06839
:10438000F701C283C0E089E00E94B90C8111C1E04D
:104390008AE00E94B90C8111C2608BE00E94B90CC6
:1043A0008111C4608CE00E94B90C8111C8608DE05D
:1043B0000E94B90C8111C0618EE00E94B90C81117C
:1043C000C0628FE00E94B90C8111C06480E10E943C
:1043D000B90C8111C068F701C383C0E081E10E947C
:1043E000B90C8111C1E082E10E94B90C8111C26057
:1043F00083E10E94B90C8111C46084E10E94B90C70
:104400008111C86085E10E94B90C8111C06186E10B
:104410000E94B90C8111C06287E10E94B90C811120
:10442000C06488E10E94B90C8111C068F701C4839F
:10443000C0E089E10E94B90C8111C1E08AE10E94CB
:10444000B90C8111C2608BE10E94B90C8111C4606A
:104450008CE10E94B90C8111C8608DE10E94B90CF9
:104460008111C0618EE10E94B90C8111C0628FE19F
:104470000E94B90C8111C06480E20E94B90C8111C4
:10448000C068F701C583CF911F91FF90EF90089509
:104490001F93CF93DF93182FEB010E943921482FF0
:1044A000833218F080E090E073C0992727E230E073
:1044B000829FB001839F700D929F700D1124FB01AC
:1044C000E759FB4F208122FD24C0FB01EB59FB4F34
:1044D0008181803F71F485859685892B39F421FD92
:1044E00005C020FD03C0878585FF03C08FE088835A
:1044F00035C0242F332787E290E0289FF001299FC1
:10450000F00D389FF00D1124EB59FB4F818188830A
:1045100025C030E0232F5EE0259FC0011124DC017F
:10452000AE5EB54FFD018181813099F490E07FE06E
:1045300060EFFD01E90FF11D8285841739F431E048
:104540008C9182FF02C0788301C068839F5F9430A2
:1045500080F32F5F253010F43323F1F2242F33271B
:1045600087E290E0289FA001299F500D389F500DB1
:104570001124FA01EB59FB4F878589838089918942
:104580009C838B83812F0E943C298A8381E090E069
:10459000DF91CF911F9108950E943921833218F045
:1045A00080E090E00895282F332787E290E0289F4D
:1045B000A001299F500D389F500D1124FA01EB598D
:1045C000FB4F8181803F59F4FA01E759FB4F20816D
:1045D00021FD05C020FD03C081E090E0089580E04A
:1045E00090E008950E943921833218F080E090E035
:1045F0000895282F332787E290E0289FA001299F64
:10460000500D389F500D1124FA01EB59FB4F2785AF
:10461000283011F0213019F481E090E0089580E015
:1046200090E00895FC018091CA099091CB09918393
:1046300080838091CC0982838091CD09838380918E
:10464000CE0984838091CF0985838091D0098683A8
:104650008091D109878308959EEF81B1892381B923
:1046600082B1892382B917B818B891EF8AB189232A
:104670008AB98BB189238BB908950F930E94392190
:10468000282F833168F000E0202F40E050E062E9FD
:104690007AE083E191E00E94462680E090E007C046
:1046A00083E999E0FC01E20FF11D808199270F91C8
:1046B00008950F930E943921833168F000E0202F84
:1046C00040E050E060EA7AE083E191E00E94462613
:1046D00080E692E212C09927880F991FFC01EB55E2
:1046E000F64F2081318184E190E0289FA001299F2D
:1046F000500D389F500D1124CA010F9108950F934A
:10470000CF93DF93EB010E943921833158F000E011
:10471000202F40E050E06FEA7AE083E191E00E94D0
:10472000462612C0992725EA39E0880F991FFC0117
:10473000E20FF31FCE0164E170E00E94A059718383
:104740006083C9010E94252CDF91CF910F910895BC
:104750000E943921833118F080E090E00895282FDD
:10476000332787E290E0289FA001299F500D389FB2
:10477000500D1124FA01EB59FB4F8089918908955E
:104780000E943921833118F080E090E00895282FAD
:10479000332787E290E0289FA001299F500D389F82
:1047A000500D1124FA01EB59FB4F85A196A10895F4
:1047B00080935E046093C90908951F93CF93C0E06E
:1047C00017E2C19FC0011124FC01EB59FB4F84A1EA
:1047D0008F3F41F00E94ED032C2F3327F901ED5656
:1047E000F64F8083CF5FC23160F383E999E00E9486
:1047F000052CCF911F910895CF9380915F04833052
:1048000059F083E080935F04C0E061E08C2F0E9448
:10481000E013CF5FC232C8F3CF91089580910B0AA5
:10482000882341F00E941B240E94462486ED99E0D3
:104830000E9493240895259A2D98269A2E988AEA04
:104840008093800089E1809381001092850010920E
:10485000840080E395E09093870080938600109217
:1048600089001092880010928B0010928A0010929A
:104870008D0010928C0060E070E081E00E94712455
:1048800060E070E082E00E94712408951092900030
:1048900084E0809391001092950010929400109201
:1048A0009700109296001092990010929800109222
:1048B0009B0010929A0010929D0010929C00109202
:1048C000D3091092D2091092D5091092D40980917F
:1048D000690088608093690010926A00E99AE19A01
:1048E000089599278230910581F0833091051CF459
:1048F000019721F00895039779F00895872F99275C
:1049000080938900609388000895872F992780936A
:104910008B0060938A000895872F992780938D00DC
:1049200060938C000895FC01118210821382128220
:1049300085E090E09583848316820895EF92FF923C
:104940000F931F93CF93DF93EC018E81982F8F5F8E
:104950008E83963068F060E375E081E00E947124F8
:1049600060E375E082E00E94712486E08E8355C08A
:104970008A819B819C0144275527888199817C01EC
:1049800000271127DA01C901689412F8880F991FCE
:10499000AA1FBB1F1694D1F7820F931FA41FB51F28
:1049A000280F391F4A1F5B1FCA01B90125E830E0F3
:1049B00040E050E00E947559A80197010E94C75934
:1049C000E901C901845490408652944010F0C0E33C
:1049D000D5E080910B0A882349F080912905803F1A
:1049E00029F4BE0181E00E94712405C060E375E0F6
:1049F00081E00E94712480910C0A882349F0809103
:104A00006106803F29F4BE0182E00E94712405C046
:104A100060E375E082E00E947124DF91CF911F91E5
:104A20000F91FF90EF9008951F920F920FB60F9283
:104A300011242F933F938F939F9380919400282F5D
:104A40003327322F2227809195009927282B392B45
:104A50008091690099278C7090700C97E1F43093E5
:104A6000D7092093D6091092940010929500809156
:104A70006304909164049093D9098093D8091092AB
:104A80006404109263041092DC09809169008B7FAA
:104A90008093690010C08091690099278C70907094
:104AA000089749F43093640420936304809169006B
:104AB0008460809369009F918F913F912F910F9017
:104AC0000FBE0F901F901895CF93DF93CDB7DEB731
:104AD00023970FB6F894DEBF0FBECDBFFE0131960F
:104AE000A0E8B1E083E090E021E08030920719F483
:104AF0000E94435A03C0182E0E94435A43E050E0DC
:104B000061E271E0CE0101960E949D48882391F0F8
:104B10000E94A425E1E2F1E0A0E8B1E083E090E0AA
:104B200021E08030920719F40E94545A03C0182ED5
:104B30000E94545A279823960FB6F894DEBF0FBEF2
:104B4000CDBFDF91CF910895CF93DF93CDB7DEB77F
:104B50006E970FB6F894DEBF0FBECDBF84E1FE01A5
:104B60003B9611928A95E9F740E064E124E130E058
:104B7000522FFE013B96469FC0011124DC01AC5729
:104B8000BE4F2115310551F081E02030380719F46E
:104B90000E94545A03C0152E0E94545AA8954F5F84
:104BA000483038F31982FE013196A3E8B1E081E084
:104BB00090E021E08030920719F40E94545A03C01B
:104BC000182E0E94545A6E960FB6F894DEBF0FBE90
:104BD000CDBFDF91CF910895CF93DF93CDB7DEB7EF
:104BE00021970FB6F894DEBF0FBECDBFFE01319600
:104BF000A3E8B1E081E090E021E08030920719F471
:104C00000E94435A03C0182E0E94435A898189305A
:104C100010F088E089838981992721960FB6F8944E
:104C2000DEBF0FBECDBFDF91CF910895CF93DF934D
:104C3000CDB7DEB764970FB6F894DEBF0FBECDBF19
:104C40009B01FE01319694E1899FD0011124A05966
:104C5000BE4F84E190E041E08030940719F40E9457
:104C6000435A03C0182E0E94435A84E1FE01319634
:104C7000D90101900D928A95E1F764960FB6F894E8
:104C8000DEBF0FBECDBFDF91CF9108956F927F92AF
:104C90008F929F92AF92BF92CF92DF92EF92FF924C
:104CA0000F931F93CF93DF93CDB7DEB7A9970FB6BE
:104CB000F894DEBF0FBECDBF6C015B013A01022F3D
:104CC000FE01B996A3E8B1E081E090E021E08030F8
:104CD000920719F40E94435A03C0182E0E94435AA7
:104CE00089A5883008F0D4C09924FE01759684E126
:104CF000DF011D928A95E9F7B601CF010E946E5936
:104D0000192D89A5981608F05EC00F2EF4E18F2E9C
:104D1000F02D0F2EF4E1EF2EFF24F02DFE01319641
:104D2000189DC0011124DC01AC57BE4FE114F10401
:104D300059F020E0E21621E0F20619F40E94435AED
:104D400003C01E2C0E94435A8D859E858A159B05A3
:104D500099F546E050E0B601CE0101960E949D48CB
:104D6000882351F5992493948F858A3008F090C058
:104D7000890D8F87053008F004E0198A1A8A1B8A8A
:104D80001C8A802F9927AC01B301CE0141960E9465
:104D90005759FE013196189DD0011124AC57BE4FD2
:104DA00084E190E021E08030920719F40E94545A87
:104DB00003C0182E0E94545A1F5F89A5181718F4B3
:104DC000992009F4ABCF992009F052C089A5883009
:104DD00008F04EC08F5F89A78CE0FE0131961192DA
:104DE0008A95E9F7F60101900020E9F731972E2F17
:104DF0002C192C3008F02BE010E0121780F4AE01D3
:104E00004F5F5F4F812F9927DC01A40FB51FF6017B
:104E1000E80FF91F80818C931F5F121798F3BE86ED
:104E2000AD8681E08F87053008F004E0088B198A91
:104E30001A8A1B8A1C8A802F9927AC01B301CE01E4
:104E400041960E945759FE01319699A584E1989F99
:104E5000D0011124A059BE4F84E190E021E08030C0
:104E6000920719F40E94545A03C0182E0E94545AF3
:104E7000FE01B996A3E8B1E081E090E021E0803046
:104E8000920719F40E94545A03C0182E0E94545AD3
:104E9000A9960FB6F894DEBF0FBECDBFDF91CF91BC
:104EA0001F910F91FF90EF90DF90CF90BF90AF9048
:104EB0009F908F907F906F900895089582E1E9E32D
:104EC000FFE011928A95E9F780E1EBE4FFE01192AF
:104ED0008A95E9F7EDE6FFE0A8E8B0E082E190E02E
:104EE00021E08030920719F40E94435A03C0182E23
:104EF0000E94435AEFE7FFE0AAE9B0E082E190E0C8
:104F000021E08030920719F40E94435A03C0182E02
:104F10000E94435AE1E9FFE0ACEAB0E080E190E0B2
:104F200021E08030920719F40E94435A03C0182EE2
:104F30000E94435AEBE5FFE0ADEBB0E082E190E088
:104F400021E08030920719F40E94435A03C0182EC2
:104F50000E94435AEEE5FAE0A5E8B0E081E090E077
:104F600021E08030920719F40E94435A03C0182EA2
:104F70000E94435AEFE5FAE0A6E8B0E082E090E054
:104F800021E08030920719F40E94435A0895182EA8
:104F90000E94435A0895CF93DF93CDB7DEB762974F
:104FA0000FB6F894DEBF0FBECDBFFE01319682E191
:104FB000DF011D928A95E9F7A8E8B0E082E190E070
:104FC00021E08030920719F40E94545A03C0182E31
:104FD0000E94545AFE013196AAE9B0E082E190E0C5
:104FE00021E08030920719F40E94545A03C0182E11
:104FF0000E94545AFE013196ACEAB0E080E190E0A4
:1050000021E08030920719F40E94545A03C0182EF0
:105010000E94545AFE013196ADEBB0E082E190E07F
:1050200021E08030920719F40E94545A03C0182ED0
:105030000E94545A0E945E2762960FB6F894DEBF13
:105040000FBECDBFDF91CF9108950E94A114982F7C
:1050500080915E0A891790F490935E0AEEE5FAE07B
:10506000A5E8B0E081E090E021E08030920719F4FB
:105070000E94545A03C0182E0E94545A0E949C1435
:105080009C0180915F0A9091600A82179307A0F4B7
:105090003093600A20935F0AEFE5FAE0A6E8B0E0FB
:1050A00082E090E021E08030920719F40E94545A87
:1050B0000895182E0E94545A089580915E0A9927E7
:1050C000089580915F0A9091600A089590E049E305
:1050D0005FE0292F3327F901E40FF51F808180FF5E
:1050E00017C08E7F8083D901A857BF4FF901E359BC
:1050F000F04F8081082E0E94485AD901A656BF4F12
:10510000F901E158F04F8081082E0E94485A089515
:10511000E92FFF27DF01A40FB51F8C9181FF0CC081
:105120008D7F8C93DF01A354BF4FE55AF04F8081F0
:10513000082E0E94485A08959F5F923150F290E0E5
:105140002BE43FE0E92FFF27DF01A20FB31F8C9173
:10515000813059F41C92DF01A455BF4FEF56F04F38
:105160008081082E0E94485A08959F5F903150F325
:105170000895282F2150223198F58DE69FE0FC01FB
:10518000E20FF11D3081832F9927929582958F70C0
:1051900089279F7089278F30910514F5482F4F5F1D
:1051A000942F9295907F832F8F70890F8083CB01EE
:1051B00083709070892B11F041E001C040E03327EB
:1051C000F901E158F04FCB01969587959695879513
:1051D000840F8083F901E75CF04F808181608083D8
:1051E0000895E82FE150E231C0F4FF27DF01A35911
:1051F000B04F2C91822F99278F7090700F971CF5CC
:10520000822F8F708F5F922F907F890F8C93E75C36
:10521000F04F80818160808308958351803198F4BC
:10522000E82FFF27DF01AF56B04F2C91822F99272F
:105230008F7090700F973CF4822F8F5F8C93E55B9B
:10524000F04F81E08083089581508231A0F4E82FEF
:10525000FF27DF01A55AB04F2C91822F99278F701D
:1052600090700F9744F4822F8F5F8C93E75CF04F20
:105270008081826080830895E82FE150E23188F4D4
:105280002E2F3327F901E359F04F8081882331F421
:10529000F901E55AF04F8081882391F081E090E098
:1052A0000895282F2351203158F481E99FE0FC0113
:1052B000E20FF11D8081882319F081E090E00895CC
:1052C00080E090E00895CF93DF93EC01FC0120E5AE
:1052D00032E08EE090E041E08030940721F4D90183
:1052E0000E94545A04C0D901182E0E94545ACE016B
:1052F0000296AC01698188810E94A514DF91CF914B
:105300000895FC01A0E5B2E08EE090E021E080305D
:10531000920719F40E94435A0895182E0E94435A86
:105320000895FC01A0E6B2E08FE190E021E080303A
:10533000920719F40E94545A0895182E0E94545A44
:105340000895FC01A0E6B2E08FE190E021E080301A
:10535000920719F40E94435A0895182E0E94435A46
:105360000895FC01A0EABBE088E090E021E08030F5
:10537000920719F40E94545A0895182E0E94545A04
:105380000895FC01A0EABBE088E090E021E08030D5
:10539000920719F40E94435A0895182E0E94435A06
:1053A00008950F93CF93DF93CDB7DEB721970FB654
:1053B000F894DEBF0FBECDBF8983853060F000E07A
:1053C00021E0AE014F5F5F4F67E470E085E291E05E
:1053D0000E94462615C0898199E1899FC001112448
:1053E000FB01DC01AE5FB04F89E190E021E080304D
:1053F000920719F40E94545A03C0182E0E94545A5E
:1054000021960FB6F894DEBF0FBECDBFDF91CF91CE
:105410000F9108950F93CF93DF93CDB7DEB7219708
:105420000FB6F894DEBF0FBECDBF8983853060F024
:1054300000E021E0AE014F5F5F4F64E570E085E280
:1054400091E00E94462615C0898199E1899FC0019B
:105450001124FB01DC01AE5FB04F89E190E021E057
:105460008030920719F40E94435A03C0182E0E94FC
:10547000435A21960FB6F894DEBF0FBECDBFDF9121
:10548000CF910F9108950F93CF93DF93CDB7DEB7F0
:1054900021970FB6F894DEBF0FBECDBF898380324F
:1054A00060F000E021E0AE014F5F5F4F60E670E02A
:1054B00085E291E00E94462614C0FB0199818CE2AE
:1054C000989FD0011124A058BC4F8CE290E021E0BD
:1054D0008030920719F40E94545A03C0182E0E947B
:1054E000545A21960FB6F894DEBF0FBECDBFDF91A0
:1054F000CF910F9108950F93CF93DF93CDB7DEB780
:1055000021970FB6F894DEBF0FBECDBF89838032DE
:1055100060F000E021E0AE014F5F5F4F6AE670E0AF
:1055200085E291E00E94462614C0FB0199818CE23D
:10553000989FD0011124A058BC4F8CE290E021E04C
:105540008030920719F40E94435A03C0182E0E941B
:10555000435A21960FB6F894DEBF0FBECDBFDF9140
:10556000CF910F9108950F93CF93DF93CDB7DEB70F
:1055700021970FB6F894DEBF0FBECDBF898384316B
:1055800060F000E021E0AE014F5F5F4F64E770E044
:1055900085E291E00E94462614C0FB01998188E1D2
:1055A000989FD0011124A05FB64F88E190E021E0E0
:1055B0008030920719F40E94545A03C0182E0E949A
:1055C000545A21960FB6F894DEBF0FBECDBFDF91BF
:1055D000CF910F9108950F93CF93DF93CDB7DEB79F
:1055E00021970FB6F894DEBF0FBECDBF89838431FB
:1055F00060F000E021E0AE014F5F5F4F6EE770E0CA
:1056000085E291E00E94462614C0FB01998188E161
:10561000989FD0011124A05FB64F88E190E021E06F
:105620008030920719F40E94435A03C0182E0E943A
:10563000435A21960FB6F894DEBF0FBECDBFDF915F
:10564000CF910F910895CF93DF93CDB7DEB76997D0
:105650000FB6F894DEBF0FBECDBFFC01862F815080
:10566000823218F080E090E02AC061508081898306
:1056700081818A8382818B8383818C8387818887E0
:105680008789888F808D898F848195819E838D8382
:1056900086818F83DF0118968FE0FE0139960D9089
:1056A00001928A95E1F789E1689FC0011124805534
:1056B000944FBC01CE0101960E94F42B9927699664
:1056C0000FB6F894DEBF0FBECDBFDF91CF91089526
:1056D0000F931F93CF93DF93CDB7DEB769970FB6C4
:1056E000F894DEBF0FBECDBF8C01962F9150923241
:1056F000B0F589E1989FC00111249E012F5F3F4FB3
:10570000DC01A055B44F89E190E041E0803094077E
:1057100021F4F9010E94435A04C0F901182E0E9495
:10572000435A8981F80180838A8181838B818283B6
:105730008C81838388858783888D878B898D808FF3
:105740008D819E81958384838F818683D80118966D
:105750008FE0FE01399601900D928A95E1F76996E6
:105760000FB6F894DEBF0FBECDBFDF91CF911F9172
:105770000F91089581508B30C8F4FB01A82FBB27EF
:10578000CD0182959295907F9827807F9827DC01A4
:10579000A051B54F80E190E021E08030920719F4EC
:1057A0000E94545A0895182E0E94545A0895815008
:1057B0008B30C8F4FB01A82FBB27CD0182959295B1
:1057C000907F9827807F9827DC01A051B54F80E11A
:1057D00090E021E08030920719F40E94435A089526
:1057E000182E0E94435A0895FC01DB0189E190E0E4
:1057F00021E08030920719F40E94545A03C0182EF9
:105800000E94545A81E090E00895FC01A0E1B0E0CC
:1058100082E190E021E08030920719F40E94545A0E
:105820000895182E0E94545A0895FC01A0E1B0E09A
:1058300082E190E021E08030920719F40E94435AFF
:105840000895182E0E94435A0895FC01A0E3B0E089
:1058500084E290E021E08030920719F40E94545ACB
:105860000895182E0E94545A0895FC01A0E3B0E058
:1058700084E290E021E08030920719F40E94435ABC
:105880000895182E0E94435A0895FC01A0E8B2E042
:1058900088E190E021E08030920719F40E94545A88
:1058A0000895182E0E94545A0895FC01A0E8B2E011
:1058B00088E190E021E08030920719F40E94435A79
:1058C0000895182E0E94435A08950F93FC01808179
:1058D000882319F488E992E016C08081813019F498
:1058E0008EED92E010C08081823019F484E293E062
:1058F0000AC000E021E0AF0167E471E085E291E0D9
:105900000E9446260DC0DC0186E490E021E0803054
:10591000920719F40E94545A03C0182E0E94545A38
:105920000F9108950F93CF93DF93CDB7DEB72197F3
:105930000FB6F894DEBF0FBECDBF8983882319F45C
:1059400088E992E018C08981813019F48EED92E0E7
:1059500012C08981823019F484E293E00CC000E027
:1059600021E0AE014F5F5F4F60E671E085E291E0BC
:105970000E9446260EC0FB01DC0186E490E021E097
:105980008030920719F40E94435A03C0182E0E94D7
:10599000435A21960FB6F894DEBF0FBECDBFDF91FC
:1059A000CF910F910895CF93DF93CDB7DEB7609776
:1059B0000FB6F894DEBF0FBECDBFFE013196A0E05A
:1059C000B0E080E190E021E08030920719F40E947D
:1059D000435A03C0182E0E94435A8B858F3119F405
:1059E0008FE190E008C08B85803219F480E290E06E
:1059F00002C08FE190E060960FB6F894DEBF0FBE54
:105A0000CDBFDF91CF910895C1EED0E1DEBFCDBF14
:105A10000E9490470E944C300E94C7140E947C054F
:105A20000E94A2470E94F23A0E946425FE0131962C
:105A3000A0E0B0E084E090E021E08030920719F42B
:105A40000E94435A03C0182E0E94435A44E050E07B
:105A500069E371E0CE0101960E949D488823C1F15F
:105A60008E010F5F1F4F8EE1D8011D928A95E9F7D5
:105A700085E0E9E3F1E0D80101900D928A95E1F724
:105A80001D821E821F82188619861A861B860E9416
:105A9000B317F801A0E0B0E080E190E021E08030B1
:105AA000920719F40E94545A03C0182E0E94545AA7
:105AB000FE013196A0E0B0E084E090E021E080308B
:105AC000920719F40E94545A03C0182E0E94545A87
:105AD000FE013196A0E3B2E08AE090E021E0803060
:105AE000920719F40E94435A03C0182E0E94435A89
:105AF0004AE050E065E571E0CE0101960E949D48C4
:105B0000882379F10E94D3170E944A0C0E94624AAE
:105B10000E9451060E94E70AFE0131968EE1DF01E4
:105B20001D928A95E9F7A2E8BFE080E190E021E0CC
:105B30008030920719F40E94545A03C0182E0E9414
:105B4000545AE5E5F1E0A0E3B2E08AE090E021E01C
:105B50008030920719F40E94545A03C0182E0E94F4
:105B6000545AFE013196A0E8B1E083E090E021E0D4
:105B70008030920719F40E94435A03C0182E0E94E5
:105B8000435A43E050E06EE371E0CE0101960E947B
:105B90009D48882391F00E94A425EEE3F1E0A0E85F
:105BA000B1E083E090E021E08030920719F40E9498
:105BB000545A03C0182E0E94545AFE013196A0E890
:105BC000B0E085E090E021E08030920719F40E9477
:105BD000435A03C0182E0E94435A45E050E062E445
:105BE00071E0CE0101960E949D48882309F475C09A
:105BF000FE0131968EE1DF011D928A95E9F7ACEB4B
:105C0000B0E081E090E021E08030920719F40E943A
:105C1000545A03C0182E0E94545AFE013196A5E82A
:105C2000B0E081E090E021E08030920719F40E941A
:105C3000545A03C0182E0E94545AFE013196A6E809
:105C4000B0E082E090E021E08030920719F40E94F9
:105C5000545A03C0182E0E94545AFE013196A8E8E7
:105C6000B0E082E190E021E08030920719F40E94D8
:105C7000545A03C0182E0E94545AFE013196ACEAC1
:105C8000B0E080E190E021E08030920719F40E94BA
:105C9000545A03C0182E0E94545AFE013196ADEB9F
:105CA000B0E082E190E021E08030920719F40E9498
:105CB000545A03C0182E0E94545AE2E4F1E0A0E8BE
:105CC000B0E085E090E021E08030920719F40E9476
:105CD000545A03C0182E0E94545AE6E2FFE0A0E78F
:105CE000B0E089E090E021E08030920719F40E9452
:105CF000435A03C0182E0E94435A8091260F909158
:105D0000270FA1E0843F9A0721F0885E934059F065
:105D100013C086E08093E20084E08093E30083E197
:105D20008093E40009C082E08093E20084E08093E5
:105D3000E30083E18093E4000E94170B8091280F19
:105D40009091290F059738F485E090E09093290F02
:105D50008093280F0DC08091280F9091290F815DAD
:105D6000974030F080ED97E09093290F8093280FB3
:105D700080912A0F90912B0FF8E080309F0738F028
:105D80008959994021F010922B0F10922A0F0E94EE
:105D90005E330E941F4A0E94F3180E94393A87E03E
:105DA0000E94D35378940E94F745A89580E00E9402
:105DB0004E3A0E94FD3AFACF1F93162FA3989927C7
:105DC00087709070880F991F81640E949B47812F74
:105DD0000E949B4780E00E949B47A39A99271F91AE
:105DE00008950F931F93162F042FA3989927877058
:105DF0009070880F991F80640E949B47812F0E949A
:105E00009B47802F0E949B47A39A1F910F91089553
:105E10001F93CF93C091610ACC2389F511E01093B1
:105E2000610A4CE16AE08C2F0E94F12E4C2F6C2FFE
:105E30008C2F0E94F12E4FEF612F8C2F0E94F12E9C
:105E40004C2F62E08C2F0E94F12E4C2F63E08C2FA0
:105E50000E94F12E4C2F64E08C2F0E94F12E4C2FCB
:105E600065E08C2F0E94F12E4C2F6CE08C2F0E944D
:105E7000F12E4C2F6DE08C2F0E94F12E0AC1C091A3
:105E8000610AC13089F54CE16AE08C2F0E94F12E45
:105E900040E0642F8C2F0E94F12E4FEF6C2F8C2F3F
:105EA0000E94F12E40E062E08C2F0E94F12E40E033
:105EB00063E08C2F0E94F12E40E064E08C2F0E9462
:105EC000F12E40E065E08C2F0E94F12E40E06CE066
:105ED0008C2F0E94F12E40E06DE08C2F0E94F12E5D
:105EE00082E08093610AD5C0C091610AC23089F511
:105EF0004CE16AE08C2F0E94F12E40E0642F8C2F41
:105F00000E94F12E4FEF61E08C2F0E94F12E40E0B5
:105F10006C2F8C2F0E94F12E40E063E08C2F0E94AA
:105F2000F12E40E064E08C2F0E94F12E40E065E00D
:105F30008C2F0E94F12E40E06CE08C2F0E94F12EFD
:105F400040E06DE08C2F0E94F12E83E08093610A87
:105F5000A0C0C091610AC33089F54CE16AE08C2F82
:105F60000E94F12E40E0642F8C2F0E94F12E4FEF03
:105F700061E08C2F0E94F12E40E062E08C2F0E94A5
:105F8000F12E40E06C2F8C2F0E94F12E40E064E057
:105F90008C2F0E94F12E40E065E08C2F0E94F12EA4
:105FA00040E06CE08C2F0E94F12E40E06DE08C2FE1
:105FB0000E94F12E84E08093610A6BC0C091610A57
:105FC000C43089F54CE16AE08C2F0E94F12E4CEF31
:105FD00060E08C2F0E94F12E4FEF61E08C2F0E9429
:105FE000F12E40E062E08C2F0E94F12E40E063E051
:105FF0008C2F0E94F12E40E06C2F8C2F0E94F12EEE
:1060000040E065E08C2F0E94F12E40E06CE08C2F88
:106010000E94F12E40E06DE08C2F0E94F12E85E071
:106020008093610A36C0C091610AC53081F54CE1A8
:106030006AE08C2F0E94F12E40E0642F8C2F0E948A
:10604000F12E40EF61E08C2F0E94F12E40E062E0E3
:106050008C2F0E94F12E40E063E08C2F0E94F12EE5
:1060600040E064E08C2F0E94F12E40E06C2F8C2FDA
:106070000E94F12E40E06CE08C2F0E94F12E40E057
:106080006DE08C2F0E94F12E1092610A02C01092D6
:10609000610ACF911F9108959B9AA39A4CE16AE0FF
:1060A00080E00E94F12E40E064E1842F0E94F12EF6
:1060B00040E0642F842F0E94F12E4FEF61E080E0DA
:1060C0000E94F12E40E062E0842F0E94F12E40E019
:1060D00063E0842F0E94F12E40E064E0842F0E9450
:1060E000F12E40E065E0842F0E94F12E40E06CE04C
:1060F000842F0E94F12E40E06DE0842F0E94F12E4B
:106100004CE16AE081E00E94F12E40E064E181E030
:106110000E94F12E40E0642F81E00E94F12E4FEFAB
:1061200061E0862F0E94F12E40E062E081E00E9453
:10613000F12E40E063E081E00E94F12E40E064E057
:1061400081E00E94F12E40E065E081E00E94F12EA6
:1061500040E06CE081E00E94F12E40E06DE081E0E3
:106160000E94F12E4CE16AE082E00E94F12E40E0B4
:1061700064E182E00E94F12E40E0642F82E00E9400
:10618000F12E4FEF61E082E00E94F12E40E062E0EC
:10619000862F0E94F12E40E063E082E00E94F12E03
:1061A00040E064E082E00E94F12E40E065E082E0A1
:1061B0000E94F12E40E06CE082E00E94F12E40E06F
:1061C0006DE082E00E94F12E4CE16AE083E00E94E3
:1061D000F12E40E064E183E00E94F12E40E0642F64
:1061E00083E00E94F12E4FEF61E083E00E94F12EE8
:1061F00040E062E083E00E94F12E40E063E0862F01
:106200000E94F12E40E064E083E00E94F12E40E025
:1062100065E083E00E94F12E40E06CE083E00E94A4
:10622000F12E40E06DE083E00E94F12E4CE16AE047
:1062300084E00E94F12E40E064E184E00E94F12EAF
:106240004CEF60E084E00E94F12E4FEF61E084E0CB
:106250000E94F12E40E062E084E00E94F12E40E0D6
:1062600063E084E00E94F12E40E064E0862F0E940B
:10627000F12E40E065E084E00E94F12E40E06CE009
:1062800084E00E94F12E40E06DE084E00E94F12E57
:106290004CE16AE085E00E94F12E40E064E185E097
:1062A0000E94F12E40E065E185E00E94F12E40E081
:1062B000642F85E00E94F12E40EF61E085E00E94AE
:1062C000F12E40E062E085E00E94F12E40E063E0C4
:1062D00085E00E94F12E40E064E085E00E94F12E0E
:1062E00040E065E0862F0E94F12E40E06CE085E002
:1062F0000E94F12E40E06DE085E00E94F12E0895AD
:106300000F931F93CF93082FC62F142F20E030E058
:10631000613611F421E030E080E090E0C13411F406
:1063200081E090E0822B932B892B91F060E0812F0C
:106330000E94DC2E21E030E0002E02C0220F331F2D
:106340000A94E2F7482F422B60E0812F0E94F12E41
:1063500020E030E0C23611F421E030E080E090E04F
:10636000C23411F481E090E0822B932B892B89F0C9
:1063700061E0812F0E94DC2E21E030E002C0220F7C
:10638000331F0A95E2F7482F422B61E0812F0E94CC
:10639000F12ECF911F910F9108950F931F93CF93DB
:1063A000082FC62F142F20E030E0613611F421E0D1
:1063B00030E080E090E0C13411F481E090E0822B85
:1063C000932B892BA1F060E0812F0E94DC2E21E02D
:1063D00030E0002E02C0220F331F0A94E2F7922F02
:1063E0009095482F492360E0812F0E94F12E20E0F4
:1063F00030E0C23611F421E030E080E090E0C234B9
:1064000011F481E090E0822B932B892B99F061E0CD
:10641000812F0E94DC2E21E030E002C0220F331FCA
:106420000A95E2F7922F9095482F492361E0812F3A
:106430000E94F12ECF911F910F9108950F931F93FA
:10644000CF93182FC62F042F20E030E0613611F4CF
:1064500021E030E080E090E0C13411F481E090E090
:10646000822B932B892B29F0412F64E1802F0E94EE
:10647000F12E20E030E0C23611F421E030E080E07F
:1064800090E0C23411F481E090E0822B932B892BB1
:1064900029F0412F65E1802F0E94F12ECF911F91AD
:1064A0000F9108950F931F93CF93082FC62F142F8A
:1064B00050E020E030E0613611F421E030E080E08F
:1064C00090E0C13411F481E090E0822B932B892B72
:1064D00071F062E1812F0E94DC2E21E030E0002E7D
:1064E00002C0220F331F0A94E2F7582F522B20E0EC
:1064F00030E0C23611F421E030E080E090E0C234B8
:1065000011F481E090E0822B932B892B69F063E1F9
:10651000812F0E94DC2E21E030E002C0220F331FC9
:106520000A95E2F7582F522B412F6C2F852F0E948E
:106530001E32CF911F910F9108950F931F93CF9308
:10654000082FC62F142F50E020E030E0613611F400
:1065500021E030E080E090E0C13411F481E090E08F
:10656000822B932B892B81F062E1812F0E94DC2EFC
:1065700021E030E0002E02C0220F331F0A94E2F720
:10658000922F9095582F592320E030E0C23611F415
:1065900021E030E080E090E0C23411F481E090E04E
:1065A000822B932B892B79F063E1812F0E94DC2EC3
:1065B00021E030E002C0220F331F0A95E2F7922F4C
:1065C0009095582F5923412F6C2F852F0E941E32F2
:1065D000CF911F910F9108951F93CF93C82F162F1E
:1065E00040E020E030E0813611F421E030E080E04E
:1065F00090E0C13411F481E090E0822B932B892B41
:1066000029F062E1812F0E94DC2E482F20E030E04B
:10661000C23611F421E030E080E090E0C23411F4A1
:1066200081E090E0822B932B892B29F063E1812F6D
:106630000E94DC2E482F842F9927CF911F91089517
:106640000F931F93CF93182FC62F042F40E020E005
:1066500030E0613611F421E030E080E090E0C134B8
:1066600011F481E090E0822B932B892B29F062E1D9
:10667000802F0E94DC2E482F20E030E0C23611F43B
:1066800021E030E080E090E0C23411F481E090E05D
:10669000822B932B892B29F063E1802F0E94DC2E23
:1066A000482F81E090E002C0880F991F1A95E2F709
:1066B00084239927CF911F910F9108950E94A30FD2
:1066C0008FEB9AE09093560B8093550B1092570BDB
:1066D00010924E0B10924F0B8EE49BE00E94AB0F7A
:1066E0008823D1F710924D0B87EC9AE09093620BC0
:1066F0008093610B1092630B10925A0B10925B0BFC
:106700008AE59BE00E94AB0F8823D1F71092590BCA
:106710008FEC9AE090936E0B80936D0B10926F0B41
:106720001092660B1092670B86E69BE00E94AB0FFF
:106730008823D1F71092650B87ED9AE090937A0B3E
:106740008093790B10927B0B1092720B1092730B4B
:1067500082E79BE00E94AB0F8823D1F71092710B68
:106760008FE69AE09093E70A8093E60A1092E80A8F
:106770001092DF0A82E08093E00A8FED9AE00E9497
:10678000AB0F8823D1F787E79AE09093F20A8093C2
:10679000F10A1092F30A1092EA0A82E08093EB0A5F
:1067A0008AEE9AE00E94AB0F8823D1F78FE79AE038
:1067B0009093FD0A8093FC0A1092FE0A1092F50A4B
:1067C00082E08093F60A85EF9AE00E94AB0F88235F
:1067D000D1F787E89AE09093080B8093070B10920B
:1067E000090B1092000B82E08093010B80E09BE08C
:1067F0000E94AB0F8823D1F78FE89AE09093130B98
:106800008093120B1092140B10920B0B82E080936A
:106810000C0B8BE09BE00E94AB0F8823D1F787E93C
:106820009AE090931E0B80931D0B10921F0B1092F9
:10683000160B82E08093170B86E19BE00E94AB0F62
:106840008823D1F78FE99AE09093290B8093280B46
:1068500010922A0B1092210B82E08093220B81E28E
:106860009BE00E94AB0F8823D1F787EA9AE09093D0
:10687000340B8093330B1092350B10922C0B82E06B
:1068800080932D0B8CE29BE00E94AB0F8823D1F705
:106890008FEA9AE090933F0B80933E0B1092400B4F
:1068A0001092370B82E08093380B87E39BE00E94C5
:1068B000AB0F8823D1F787EB9AE090934A0B809334
:1068C000490B10924B0B1092420B82E08093430BCA
:1068D00082E49BE00E94AB0F8823D1F7089580915A
:1068E0004D0B8823E1F080914D0B813059F48DE4FC
:1068F0009BE001960E94AB0F882389F482E080938D
:106900004D0B0DC080914D0B823049F48DE49BE01E
:1069100001960E94BD10882311F480934D0B809145
:10692000590B8823E1F08091590B813059F489E5A6
:106930009BE001960E94AB0F882389F482E080934C
:10694000590B0DC08091590B823049F489E59BE0C9
:1069500001960E94BD10882311F48093590B8091F9
:10696000650B8823E1F08091650B813059F485E651
:106970009BE001960E94AB0F882389F482E080930C
:10698000650B0DC08091650B823049F485E69BE074
:1069900001960E94BD10882311F48093650B8091AD
:1069A000710B8823E1F08091710B813059F481E7FC
:1069B0009BE001960E94AB0F882389F482E08093CC
:1069C000710B08958091710B823049F481E79BE04F
:1069D00001960E94BD10882311F48093710B0895D5
:1069E000CF93DF93EC018FED9AE00E94BD108823D6
:1069F00009F046C08091E10A9091E20AAA27BB27DC
:106A000088839983AA83BB83E091E60AF091E70A21
:106A100080818D83E091E60AF091E70A81818E837F
:106A2000E091E60AF091E70A82818F83E091E60A1D
:106A3000F091E70A83818887E091E60AF091E70AFE
:106A400084818987E091E60AF091E70A85818A8747
:106A5000E091E60AF091E70A86818B87E091E60AE9
:106A6000F091E70A87818C878091E50A8C838FED0E
:106A70009AE00E94AB0F8823D1F781E090E0BBC27F
:106A80008AEE9AE00E94BD10882309F046C08091EA
:106A9000EC0A9091ED0AAA27BB2788839983AA83E1
:106AA000BB83E091F10AF091F20A80818D83E0913D
:106AB000F10AF091F20A81818E83E091F10AF0915E
:106AC000F20A82818F83E091F10AF091F20A8381C8
:106AD0008887E091F10AF091F20A84818987E09138
:106AE000F10AF091F20A85818A87E091F10AF0912A
:106AF000F20A86818B87E091F10AF091F20A878190
:106B00008C878091F00A8C838AEE9AE00E94AB0F0A
:106B10008823D1F781E090E06EC285EF9AE00E9471
:106B2000BD10882309F046C08091F70A9091F80AB9
:106B3000AA27BB2788839983AA83BB83E091FC0A99
:106B4000F091FD0A80818D83E091FC0AF091FD0AAD
:106B500081818E83E091FC0AF091FD0A82818F830E
:106B6000E091FC0AF091FD0A83818887E091FC0A9C
:106B7000F091FD0A84818987E091FC0AF091FD0A79
:106B800085818A87E091FC0AF091FD0A86818B87D6
:106B9000E091FC0AF091FD0A87818C878091FB0AC5
:106BA0008C8385EF9AE00E94AB0F8823D1F781E0B8
:106BB00090E021C280E09BE00E94BD10882309F094
:106BC00046C08091020B9091030BAA27BB278883B4
:106BD0009983AA83BB83E091070BF091080B808116
:106BE0008D83E091070BF091080B81818E83E091FA
:106BF000070BF091080B82818F83E091070BF091D6
:106C0000080B83818887E091070BF091080B848142
:106C10008987E091070BF091080B85818A87E091C5
:106C2000070BF091080B86818B87E091070BF091A1
:106C3000080B87818C878091060B8C8380E09BE01A
:106C40000E94AB0F8823D1F781E090E0D4C18BE0A4
:106C50009BE00E94BD10882309F046C080910D0B77
:106C600090910E0BAA27BB2788839983AA83BB83A5
:106C7000E091120BF091130B80818D83E091120B48
:106C8000F091130B81818E83E091120BF091130B25
:106C900082818F83E091120BF091130B838188879F
:106CA000E091120BF091130B84818987E091120B14
:106CB000F091130B85818A87E091120BF091130BF1
:106CC00086818B87E091120BF091130B87818C8763
:106CD0008091110B8C838BE09BE00E94AB0F88238B
:106CE000D1F781E090E087C186E19BE00E94BD1072
:106CF000882309F046C08091180B9091190BAA27A0
:106D0000BB2788839983AA83BB83E0911D0BF091F5
:106D10001E0B80818D83E0911D0BF0911E0B8181F4
:106D20008E83E0911D0BF0911E0B82818F83E09189
:106D30001D0BF0911E0B83818887E0911D0BF09154
:106D40001E0B84818987E0911D0BF0911E0B8581BC
:106D50008A87E0911D0BF0911E0B86818B87E09155
:106D60001D0BF0911E0B87818C8780911C0B8C83EF
:106D700086E19BE00E94AB0F8823D1F781E090E091
:106D80003AC181E29BE00E94BD10882309F046C011
:106D90008091230B9091240BAA27BB27888399838A
:106DA000AA83BB83E091280BF091290B80818D830E
:106DB000E091280BF091290B81818E83E091280BC3
:106DC000F091290B82818F83E091280BF091290BA0
:106DD00083818887E091280BF091290B8481898732
:106DE000E091280BF091290B85818A87E091280B8F
:106DF000F091290B86818B87E091280BF091290B6C
:106E000087818C878091270B8C8381E29BE00E9495
:106E1000AB0F8823D1F781E090E0EDC08CE29BE0DE
:106E20000E94BD10882309F046C080912E0B9091DE
:106E30002F0BAA27BB2788839983AA83BB83E09162
:106E4000330BF091340B80818D83E091330BF09103
:106E5000340B81818E83E091330BF091340B82816E
:106E60008F83E091330BF091340B83818887E0911D
:106E7000330BF091340B84818987E091330BF091CF
:106E8000340B85818A87E091330BF091340B868136
:106E90008B87E091330BF091340B87818C87809145
:106EA000320B8C838CE29BE00E94AB0F8823D1F7DE
:106EB00081E090E0A0C087E39BE00E94BD108823A2
:106EC00009F046C08091390B90913A0BAA27BB2755
:106ED00088839983AA83BB83E0913E0BF0913F0B9B
:106EE00080818D83E0913E0BF0913F0B81818E83F9
:106EF000E0913E0BF0913F0B82818F83E0913E0B3E
:106F0000F0913F0B83818887E0913E0BF0913F0B1E
:106F100084818987E0913E0BF0913F0B85818A87C0
:106F2000E0913E0BF0913F0B86818B87E0913E0B09
:106F3000F0913F0B87818C8780913D0B8C8387E399
:106F40009BE00E94AB0F8823D1F781E090E053C013
:106F500082E49BE00E94BD10882309F046C0809126
:106F6000440B9091450BAA27BB2788839983AA835A
:106F7000BB83E091490BF0914A0B80818D83E091B6
:106F8000490BF0914A0B81818E83E091490BF0917E
:106F90004A0B82818F83E091490BF0914A0B8381E8
:106FA0008887E091490BF0914A0B84818987E091B1
:106FB000490BF0914A0B85818A87E091490BF0914A
:106FC0004A0B86818B87E091490BF0914A0B8781B0
:106FD0008C878091480B8C8382E49BE00E94AB0FEE
:106FE0008823D1F781E090E006C0188219821A82C6
:106FF0001B8280E090E0DF91CF910895CF93DF93E3
:10700000DC0180914D0B882339F48DE49BE0909353
:107010007E0B80937D0B21C08091590B882339F41E
:1070200089E59BE090937E0B80937D0B16C0809149
:10703000650B882339F485E69BE090937E0B809363
:107040007D0B0BC08091710B882309F072C081E722
:107050009BE090937E0B80937D0BE0917D0BF091F4
:107060007E0B0084F185E02DED018D818083E09120
:107070007D0BF0917E0B0084F185E02D8E81818364
:10708000E0917D0BF0917E0B0084F185E02D8F81E6
:107090008283E0917D0BF0917E0B0084F185E02DE1
:1070A00088858383E0917D0BF0917E0B0084F185D0
:1070B000E02D89858483E0917D0BF0917E0B008427
:1070C000F185E02D8A858583E0917D0BF0917E0B23
:1070D0000084F185E02D8B858683E0917D0BF09116
:1070E0007E0B0084F185E02D8C858783E0917D0BFC
:1070F000F0917E0B8C818783E0917D0BF0917E0B6C
:107100008D919C9194838383E0917D0BF0917E0B14
:107110001286E0917D0BF0917E0B1182E0917D0B48
:10712000F0917E0B1282E0917D0BF0917E0B81E05D
:107130008083DF91CF91089582E69AE00E94F03437
:10714000882361F182E69AE00E94500D82E69AE07F
:107150000E94F034882311F182E69AE00E94500DDB
:1071600082E69AE00E94F0348823C1F082E69AE039
:107170000E94500D82E69AE00E94F034882371F05C
:1071800082E69AE00E94500D82E69AE00E94F03476
:10719000882321F082E69AE00E94500D0895FF9224
:1071A0000F931F93CF93DF93CDB7DEB760970FB6E2
:1071B000F894DEBF0FBECDBF20E0822F9927880F45
:1071C000991F880F991F8C010158144FF8011082E4
:1071D000F22EF394BE016F5F7F4F8F2D0E94D72B4D
:1071E0008889F8018283138211822F2D2B3028F396
:1071F00060960FB6F894DEBF0FBECDBFDF91CF9182
:107200001F910F91FF900895FC01808199270097AD
:1072100019F0019731F0089582E0838381E0808343
:1072200008958381882389F48281882329F481E069
:10723000818382E0808308958181813011F41182FD
:1072400002C081E0818382E080830895FC01808117
:107250009927813091059CF0833091051CF00397AC
:1072600031F0089582E0838383E0808308958381F1
:10727000882329F480838281882309F481830895F7
:1072800020E0822F9927880F991F880F991FFC01F2
:10729000E158F44F8381882311F0815083832F5F5D
:1072A0002B3078F3EFE7FBE0309B04C0CF010E9466
:1072B000043903C0CF010E942639E3E8FBE031998D
:1072C00004C0CF010E94043903C0CF010E942639B7
:1072D000E7E8FBE0329904C0CF010E94043903C003
:1072E000CF010E942639EBE8FBE0499904C0CF01A9
:1072F0000E94043903C0CF010E942639EFE8FBE069
:10730000349904C0CF010E94043903C0CF010E9408
:107310002639E3E9FBE0359904C0CF010E94043926
:1073200003C0CF010E942639E7E9FBE0369904C08B
:10733000CF010E94043903C0CF010E942639EBE936
:10734000FBE0379904C0CF010E94043903C0CF018C
:107350000E942639EFE9FBE0339904C0CF010E9477
:10736000043903C0CF010E942639E3EAFBE04A99C1
:1073700004C0CF010E94043903C0CF010E94263906
:10738000E7EAFBE04B9904C0CF010E94043908955D
:10739000CF010E94263908959927853C910509F46B
:1073A0003FC0863C9105A4F4823C910569F1833C81
:1073B00091053CF4803C9105F9F0813C910501F187
:1073C00047C0833C9105C1F1843C910529F140C03F
:1073D000813D9105E9F0823D91053CF4863C9105A3
:1073E00019F1873C910521F133C0823D910541F1AE
:1073F000833D910549F12CC08091800B9927089518
:107400008091840B992708958091880B992708957E
:1074100080918C0B992708958091900B992708955E
:107420008091940B992708958091980B992708953E
:1074300080919C0B992708958091A00B992708951E
:107440008091A40B992708958091A80B99270895FE
:107450008EEF90E008951092B60087E08093B00020
:107460001092B2008EE48093B30082E080937000AB
:1074700008950E942B3A1092AD0B1092AE0B109211
:10748000AF0B1092B00B1092B50B1092B60B0E947E
:10749000CF380E94FA050E945E270895CF93C82F27
:1074A0008091AB0B882311F01092AB0BA8950E9432
:1074B0009C38C23011F00E946F34C23009F46FC0A2
:1074C0008091AC0B882309F444C08091AC0B8150AF
:1074D0008093AC0B8091AD0B8F5F8093AD0B8230AE
:1074E00040F01092AD0B0E9440390E946E110E9434
:1074F00034078091AE0B8F5F8093AE0B843040F0E9
:107500001092AE0B0E94E3110E94964A0E94AF4770
:107510008091AF0B8F5F8093AF0B8A3030F0109269
:10752000AF0BC13011F00E94380D8091B00B8F5F0E
:107530008093B00B843168F01092B00B8091B50B42
:107540008F5F8093B50B0E94082F0E943C120E940F
:10755000E70C8091B50B8A3010F11092B50B809139
:10756000B10B9091B20BA091B30BB091B40B0196FB
:10757000A11DB11D8093B10B9093B20BA093B30BDF
:10758000B093B40B0E9466288091B60B8F5F8093F6
:10759000B60B8C3320F01092B60B0E942528CF91A9
:1075A00008958091B10B9091B20BA091B30BB09163
:1075B000B40BBC01CD0108951F920F920FB60F922C
:1075C00011248F931092B20081E08093AB0B8091D5
:1075D000AC0B8F5F8093AC0B8F910F900FBE0F9011
:1075E0001F9018950E944E460E94014860E076E97F
:1075F00080E090E00E941C48089504C00E949446D8
:107600000E94E7460E947E468823C1F70895FC0148
:1076100090E061506F3F21F0819198276150E0F731
:10762000892F992708950F931F938C01FC01818165
:107630008150682FC80101960E94073BF8018083A2
:1076400081819927BC01C8010E94AF461F910F910B
:107650000895AF92BF92CF92DF92EF92FF920F9375
:107660001F93CF93DF93CDB7DEB7C35ED0400FB685
:10767000F894DEBF0FBECDBF6C01FC01818181504B
:10768000682FC60101960E94073BD6019C9198176E
:1076900011F00C94DC45F6018281882309F0F8C0D2
:1076A000838199278135910509F449C08235910577
:1076B0003CF48033910589F08035910561F1E8C093
:1076C0008335910509F48EC0833591050CF478C09B
:1076D0008435910509F4B2C0DBC08E01035D1F4FF4
:1076E00080E5D8011D928A95E9F785E18EA71FA64E
:1076F00080E888ABF601848189AB992796012B5FDE
:107700003F4FAC01B901CE01C2960E945759C80142
:107710000E94133BBDC08E01035D1F4F80E5D80161
:107720001D928A95E9F785E08EA71FA680EA88ABAF
:107730000E94EC2589ABC8010E94133BA9C0F60149
:10774000B4800F2EFDE2EF2EFF24F02DEC0EFD1E77
:1077500080E5D7011D928A95E9F789E18EA71FA6DA
:1077600081EA88AB8E0103581F4FB8018B2D0E9410
:107770001626B9AA8CE0FE01F296D8010D9001926E
:107780008A95E1F7F801848595859FAF8EAF868550
:10779000FE01E05CFF4F8083F8018785FE01EF5B0F
:1077A000FF4F80839927AC01BE0163577F4FCE0105
:1077B0008E5B9F4F0E945759C7010E94133B68C0C0
:1077C0000E94A425FE01BD9680E5DF011D928A95E9
:1077D000E9F784E08EA71FA682EA88ABCF010E945A
:1077E000133B56C0F601458156818481FE01ED515F
:1077F000FF4F8083813108F04BC080E5FE01BD96CC
:1078000011928A95E9F787E18EA71FA683EA88ABD4
:107810005BAB4AABFE01ED51FF4F808189ABFE01AE
:10782000F4969927DA01019724F00E943B5A0192BD
:10783000FACFCE018D960E94133B2AC0F6014581F6
:1078400056818481FE01ED51FF4F8083813100F527
:10785000F60137969927DA01019724F001900E94EA
:10786000485AFACFDE019D9680E5FD0111928A9576
:10787000E9F787E08EA71FA684EA88AB5BAB4AAB2B
:10788000FE01ED51FF4F808189ABCD010E94133B7A
:10789000F6018281813011F00C94E54583819927AE
:1078A000AA27BB27FC013197E736F10510F00C94AD
:1078B000CE45E65BFF4FEE0FFF1F0590F491E02DE4
:1078C00009940E94FC23F601B4808B2D81508232F2
:1078D00010F00C94E54520E0AE01475F5F4F822F2A
:1078E0009927DA01A80FB91FF601E80FF91F828561
:1078F0008C932F5F2F3098F3F601858189838681E1
:107900008A8387818B83838D948D9E838D83858DE0
:107910008F838085888781858C83818D888F828DF8
:10792000898F6B2DCE0101960E94232B6B2DCE01EA
:1079300001960E949F191DA685E08EA711E01FA742
:1079400081E888AB19AACE018D960E94133B812F46
:107950000E944E3A0C94E545F601B4808B2D81507F
:10796000823208F047C06B2DCE0101960E94682B31
:107970008EE18EA781E08FA782E888ABB9AA8981C2
:107980008AAB8A818BAB8B818CAB8C818EAB8D81EA
:107990009E81FE01E85BFF4F918380838F81FE0112
:1079A000E65BFF4F808320E0BE016F5F7F4FAE013B
:1079B000475F5F4F822F9927DC01A60FB71FFA019F
:1079C000E80FF91F8081FD0186AB2F5F2F3090F308
:1079D00088858DAB888DFE01EA5BFF4F8083898DA2
:1079E000FE01E95BFF4F8083CE018D960E94133B21
:1079F0000C94E545FFEFBF1611F00C94E545FE0130
:107A0000ED51FF4F1082FE01ED51FF4F8081982F05
:107A1000823210F00C94E5450F2EF3EEEF2EFF248A
:107A2000F02DEC0EFD1E6E010894C11CD11C8E01C0
:107A3000075F1F4F892F8F5F682FCE0101960E942D
:107A4000682B8EE18EA781E08FA782E888ABD701F3
:107A50008C918F5F89AB89818AAB8A818BAB8B815B
:107A60008CAB8C818EAB8D819E81FE01E85BFF4FDC
:107A7000918380838F81FE01E65BFF4F808320E04E
:107A8000822F9927DC01AC0DBD1DF801E80FF91F0D
:107A90008081FD0186AB2F5F2F3090F388858DAB01
:107AA000888DFE01EA5BFF4F8083898DFE01E95BD3
:107AB000FF4F8083CE018D960E94133B81E00E9490
:107AC0004E3AD7018C918F5F8C93982F823208F4B5
:107AD000B1CF0C94E5450E94FC23F601B480AE01C1
:107AE00043585F4F96012B5F3F4F8FE0DA01F9015A
:107AF00001900D928A95E1F7F6018489FA01878752
:107B0000BA018B2D0E94BA2B81E08FA783E888AB46
:107B1000B9AA85E08EA7CE018D960E94133B0C94E6
:107B2000E545F601B4808B2D81508A3010F581E057
:107B30008FA784E888ABB9AA8E0103581F4FB801FC
:107B40008B2D0E94D72B8FE0FE01F296D8010D906D
:107B500001928A95E1F7F8018785FE01EF5BFF4FFF
:107B6000808385E18EA7CE018D960E94133B0C94F5
:107B7000E545FFEFBF1611F00C94E545FE01ED5110
:107B8000FF4F1082FE01ED51FF4F8081982F8B3007
:107B900010F00C94E545BB24B3948E0103581F4F9D
:107BA0000F2EFFE0AF2EF02D0F2EF1E4EF2EFF246D
:107BB000F02DEC0EFD1E0F2EF3EECF2EDD24F02D5A
:107BC000CC0EDD1EBFA684E888AB892F8F5F89AB02
:107BD000B8010E94D72BFE01F296D8012A2D0D90F4
:107BE00001922A95E1F7F8018785D7018C9385E109
:107BF0008EA7CE018D960E94133B8B2D0E944E3A8C
:107C0000F60180818F5F8083982F8B30D8F2DDC79B
:107C10000E94FC230E94C714A8950E94D317A89520
:107C20000E94F318A8950E944A0CA8950E94624AE7
:107C3000A8950E945106A8950E94CB270E94E70AAA
:107C400081E08FA786E888AB84E08EA7CE018D9671
:107C50000E94133BBAC784E18EA781E08FA787E813
:107C600088AB8DE0A8E4B1E0FE01F1960D900192A1
:107C70008A95E1F70E94D13A9B01AC01AA27BB2764
:107C80008EAFBB27A52F942F832F8FAFFE01E05C13
:107C9000FF4F2083CE018D960E94133B96C70C9414
:107CA000000093C7C60104960E94B12981E08FA706
:107CB00089E888AB84E08EA7CE018D960E94133BA5
:107CC00084C781E08FA78AE888AB8CE08EA7CE01BD
:107CD000C1960E94C129CE018D960E94133B75C7A3
:107CE000CE0187960E94562181E08FA781EA88AB5A
:107CF0008FA189AB88A58AAB89A58BAB8AA58CABF4
:107D00008BA58DAB8CA58EAB8AE08EA7CE018D9610
:107D10000E94133B5AC7F601B480F1E2FB15F8F05C
:107D2000BE016E5D7F4F8B2D0E94482281E08FA7A0
:107D300082EA88ABB9AA8BA18BAB8CA18EAB8AA14E
:107D40008AAB8DA19EA1892F99278CAB8DA18DAB7C
:107D50008AE08EA7CE018D960E94133B36C72FEF87
:107D6000B21609F032C7FE01ED51FF4F1082FE013D
:107D7000ED51FF4F8081982F823208F026C7FF24F3
:107D8000F3948F01BE016E5D7F4F892F8F5F0E943C
:107D90004822FFA682EA88ABD8018C918F5F89AB1D
:107DA0008BA18BAB8CA18EAB8AA18AAB8DA19EA13E
:107DB000892F99278CAB8DA18DAB8AE08EA7CE0140
:107DC0008D960E94133B8F2D0E944E3AF8018081C0
:107DD0008F5F8083982F8232A8F2F7C6CE014A9631
:107DE0000E9412238AE08EA781E08FA780EA88ABE9
:107DF00088A189AB8E8D8AAB8A8D9B8D892F99271F
:107E00008BAB8A8D8CAB8D8D8DAB8C8D8EABCE017B
:107E10008D960E94133BD9C6F601648180E00E94D2
:107E2000941B84E08EA781E08FA783EA88ABCE0104
:107E30008D960E94133BC9C6DE01A353BF4FF601C6
:107E400084818C938581FD018183F6018681FD010A
:107E50008283F6018781FD018383F6018085FD0120
:107E60008483F6018185FD018583F6018285FD010C
:107E70008683F6018385FD018783CD010E949C1BCB
:107E800084E08EA781E08FA784EA88ABCE018D962F
:107E90000E94133B9AC6FE01E358FF4FA0E0B0E0FA
:107EA00080E190E021E08030920719F40E94435A6B
:107EB00003C0182E0E94435AF60184819581A68141
:107EC000B781FE01EF57FF4F80839183A283B38375
:107ED000DE01A358BF4FF6018085FD018087F601C2
:107EE0008185FD018187F6018285FD018287A0E001
:107EF000B0E080E190E021E08030920719F40E9428
:107F0000545A03C0182E0E94545A84E08EA781E070
:107F10008FA780EC88ABCE018D960E94133B55C68F
:107F2000FE01E358FF4FA0E0B0E080E190E021E0E7
:107F30008030920719F40E94435A03C0182E0E9401
:107F4000435A8BE08EA781E08FA781EC88ABFE01BE
:107F5000EF57FF4F80819181A281B38189AB9AABAA
:107F6000ABABBCABFE01E358FF4F80858DAB818589
:107F70008EAB82858FABCE018D960E94133B25C6BA
:107F80008AE38EA781E08FA780ED88ABFE01F19692
:107F9000A8E8B0E082E190E021E08030920719F497
:107FA0000E94435A03C0182E0E94435AFE01ED5B03
:107FB000FF4FAAE9B0E082E190E021E08030920733
:107FC00019F40E94435A03C0182E0E94435AFE011E
:107FD000EB5AFF4FADEBB0E082E190E021E0803062
:107FE000920719F40E94435A03C0182E0E94435A64
:107FF000CE018D960E94133BE8C584E18EA781E0F7
:108000008FA78EED88ABFE01F196ACEAB0E080E17F
:1080100090E021E08030920719F40E94435A03C097
:10802000182E0E94435ACE018D960E94133BCDC557
:108030000E94CB2784E08EA781E08FA781ED88ABDB
:10804000CE018D960E94133BC0C588E08EA781E0CB
:108050008FA78FED88AB0E945D288BAB0E946128B3
:108060009AAB89ABFE01ED51FF4FACEBB0E081E084
:1080700090E021E08030920719F40E94435A03C037
:10808000182E0E94435AFE01ED51FF4F80818CABA8
:10809000CE018D960E94133B98C5FE01E358FF4F19
:1080A00080E5DF011D928A95E9F7ACEBB0E081E055
:1080B00090E021E08030920719F40E94545A03C0E6
:1080C000182E0E94545AFE01E358FF4FA5E8B0E075
:1080D00081E090E021E08030920719F40E94545A28
:1080E00003C0182E0E94545AFE01E358FF4FA6E821
:1080F000B0E082E090E021E08030920719F40E9425
:10810000545A03C0182E0E94545A84E08EA781E06E
:108110008FA780EE88ABCE018D960E94133B55C58C
:10812000F601858196819093270F8093260F878192
:1081300090859093290F8093280F81859285909345
:108140002B0F80932A0F838580932C0F8485809337
:108150002D0F858580932E0FE6E2FFE0A0E7B0E0CB
:1081600089E090E021E08030920719F40E94545A8F
:1081700003C0182E0E94545A85E08EA791E09FA755
:1081800085EA88AB99ABCE018D960E94133B1DC545
:108190008EE08EA781E08FA786EA88AB19AA80912E
:1081A000E200863069F48091E300843049F48091E4
:1081B000E400833129F484EF91E09BAB8AAB13C0D8
:1081C0008091E200823069F48091E300843049F4C8
:1081D0008091E400833129F488EE93E09BAB8AAB75
:1081E00002C01BAA1AAA8091280F9091290F9DAB5B
:1081F0008CAB80912A0F90912B0F9FAB8EAB80910F
:108200002C0F88AF80912D0F89AF80912E0F8AAFF0
:10821000CE018D960E94133BD8C4DE01AB52BF4FF6
:10822000F60184818C938581FD018183D6011696A8
:108230008CE0FE01E952FF4F0D9001928A95E1F723
:10824000FE01ED51FF4F1082FE01ED51FF4F808185
:10825000982F8C30A0F49E012B523F4FDF01F90183
:10826000E90FF11D8281882321F08F3F11F08150A9
:1082700082838C918F5F8C93982F8C3080F3CE010A
:108280008B529F4F0E94632984E08EA781E08FA7C5
:1082900087EA88ABCE018D960E94133B96C48E016F
:1082A0000B521F4FC8010E94812982E18EA781E0F5
:1082B0008FA788EA88ABD8018C9189ABF8018181BE
:1082C0008AABFE01ED51FF4F1082FE01ED51FF4FD1
:1082D0008081982F8C3080F49801DF01F901E90F3B
:1082E000F11D82818F3F11F08F5F82838C918F5FB0
:1082F0008C93982F8C3090F38CE0DE01A952BF4F05
:10830000FE01F3960D9001928A95E1F7CE018D96CC
:108310000E94133B5AC4F6018481FE01E358FF4FCB
:108320008083D60115968EE0FE01E258FF4F0D9036
:1083300001928A95E1F7FE01ED51FF4F1082FE0197
:10834000ED51FF4F8081982F8E30A0F49E0123586D
:108350003F4FDF01F901E90FF11D8181882321F0F1
:108360008F3F11F0815081838C918F5F8C93982F78
:108370008E3080F3DE01A358BF4FF6018389FD01E3
:108380008787F6018489FD01808BD60155968EE0A2
:10839000FE01E257FF4F0D9001928A95E1F7FE0131
:1083A000ED51FF4F1082FE01ED51FF4F8081982F5C
:1083B0008E30A0F49E0123583F4FDF01F901E90FF1
:1083C000F11D8189882321F08F3F11F08150818B2D
:1083D0008C918F5F8C93982F8E3080F3CE018358D1
:1083E0009F4F0E94912984E08EA781E08FA789EAA0
:1083F00088ABCE018D960E94133BE7C38E010358D4
:108400001F4FC8010E94A12983E28EA781E08FA798
:108410008AEA88ABD8018C9189ABFE01ED51FF4F00
:108420001082FE01ED51FF4F8081982F8E3080F435
:108430009801DF01F901E90FF11D81818F3F11F0F2
:108440008F5F81838C918F5F8C93982F8E3090F308
:108450008EE0DE01A258BF4FFE01F2960D90019210
:108460008A95E1F7DE01A358BF4FFD018785FE0124
:10847000E05CFF4F8083FD018089FE01EF5BFF4FD1
:108480008083FE01ED51FF4F1082FE01ED51FF4F41
:108490008081982F8E3080F49D01DF01F901E90F72
:1084A000F11D81898F3F11F08F5F818B8C918F5FE0
:1084B0008C93982F8E3090F38EE0DE01A257BF4F41
:1084C000FE01EE5BFF4F0D9001928A95E1F7CE0120
:1084D0008D960E94133B79C3F601B480858199275C
:1084E000982F88272681820F911DBC018B2D0E9419
:1084F0007F2385E08EA781E08FA782EC88ABB9AAA5
:10850000CE018D960E94133B60C3F601B4808CE0CF
:108510008EA781E08FA783EC88ABB9AA8B2D0E9430
:108520003D238AAB8B2D0E945923892F99278BAB32
:108530008B2D0E9459238CAB8B2D0E94A823892F51
:1085400099278DAB8B2D0E94A8238EAB8B2D0E947B
:10855000C023892F99278FAB8B2D0E94C02388AF12
:10856000CE018D960E94133B30C320E0F60184813A
:1085700081FD21E0F601848182FD2260F601818186
:10858000863029F46581822F0E94D8231EC360E0C3
:10859000822F0E94D82319C30E94DD2384E08EA776
:1085A00081E08FA785EC88ABCE018D960E94133BAE
:1085B0000CC3F601B4809E0123583F4F9581492F8B
:1085C0004170D9018C91887F9670842B892B8C9374
:1085D00086819781F90192838183F6018085918557
:1085E000F90194838383F6018685F9018187F60179
:1085F0008785F9018287F60182859385F901968343
:108600008583F60184859585F90190878783F60136
:108610008089F9018387F6018189F9018487F60150
:108620008289F9018587F6018389F9018687D60158
:1086300054968FE0FE01E457FF4F0D9001928A950A
:10864000E1F7F60183A1F901868FF60184A1F90112
:10865000878FF60185A1F90180A3F60186A1F901B2
:1086600081A315E0D6019796FE01E156FF4F812FB9
:108670000D9001928A95E1F7F60184A595A5A6A52E
:10868000B7A5F90187A390A7A1A7B2A7F60180A972
:10869000F90183A7B9018B2D0E94432A81E08FA79E
:1086A00082ED88AB1EA7B9AACE018D960E94133B1E
:1086B0008CC2F601B4808E0103581F4FB8018B2D78
:1086C0000E947B2A81E08FA783ED88AB81E38EA790
:1086D000B9AAD8019C91292F21708AA9887F967008
:1086E000822B892B8AABF801818192819CAB8BAB69
:1086F000838194819EAB8DAB81858BAF82858CAF5E
:108700008581968198AF8FAB878190859AAF89AF2D
:1087100083858DAF84858EAF85858FAF8685FE017D
:10872000E05CFF4F80838FE0DE01A457BF4FFE0166
:10873000EF5BFF4F0D9001928A95E1F7F801868D6E
:10874000FE01E05BFF4F8083F801878DFE01EF5A49
:10875000FF4F8083F80180A1FE01EE5AFF4F808316
:10876000F80181A1FE01ED5AFF4F808385E0DE0113
:10877000A156BF4FFE01EC5AFF4F0D9001928A9512
:10878000E1F7F80187A190A5A1A5B2A5FE01E75ADE
:10879000FF4F80839183A283B383F80183A5FE01F9
:1087A000E35AFF4F8083CE018D960E94133B0DC28A
:1087B000F601B480AE0143585F4F828DDA018C938D
:1087C000838DFA018183F601848DFA018283F6019B
:1087D0008681FA018383F6018781FA018483F60199
:1087E0008085FA018583F6018185FA018683F60189
:1087F0008285FA018783F601858DFA01878BC60190
:108800000B962FE0FE01EB57FF4FDC010D9001921C
:108810002A95E1F7BA018B2D0E94B32A81E08FA738
:1088200084ED88AB85E08EA7B9AACE018D960E9413
:10883000133BCBC1F601B4808E0103581F4FB80122
:108840008B2D0E94EB2A81E08FA785ED88AB8FE10D
:108850008EA7B9AAD8018C91FE01E95BFF4F8083F6
:10886000F8018181FE01E85BFF4F8083F80182817E
:10887000FE01E75BFF4F8083F80183818BAB84812E
:108880008CAB85818DAB86818EAB87818FAB8789E1
:10889000FE01E65BFF4F80838FE0DE01AB57BF4FE9
:1088A000FE01F8960D9001928A95E1F7CE018D9622
:1088B0000E94133B8AC1F6013496A0E0B9E080E142
:1088C00090E021E08030920719F40E94545A03C0CE
:1088D000182E0E94545A81E08FA783EE88AB84E063
:1088E0008EA7CE018D960E94133B6FC181E08FA7AA
:1088F00084EE88AB84E18EA7FE01F196A0E0B9E09A
:1089000080E190E021E08030920719F40E94435A00
:1089100003C0182E0E94435ACE018D960E94133B2D
:1089200054C1F601B480C6010596BC018B2D0E948E
:10893000D12981E08FA788ED88AB85E08EA7B9AA01
:10894000CE018D960E94133B40C1F601B48081E0B8
:108950008FA789ED88AB8EE18EA7B9AABE016E5CA8
:108960007F4F8B2D0E940A2ACE018D960E94133BC9
:108970002CC1F60184818093300F85818093310F63
:1089800086818093320F87818093330F8085809317
:10899000340F81858093350F82858093360F8385D0
:1089A0008093370FE0E3FFE0A2E9BFE088E090E0CA
:1089B00021E08030920719F40E94545A03C0182E07
:1089C0000E94545A81E08FA785EE88AB84E08EA781
:1089D000CE018D960E94133BF8C081E08FA786EEF2
:1089E00088AB8CE08EA78091300F89AB8091310FDE
:1089F0008AAB8091320F8BAB8091330F8CAB80911F
:108A0000340F8DAB8091350F8EAB8091360F8FABCD
:108A10008091370F88AFCE018D960E94133BD5C051
:108A2000C60105960E94452C81E08FA786ED88AB94
:108A300085E08EA7CE018D960E94133BC6C081E0D3
:108A40008FA787ED88AB8DE18EA7CE01C2960E94DD
:108A5000552CCE018D960E94133BB7C0F601B48011
:108A6000C60104960E94652C81E08FA78AED88AB31
:108A700085E08EA7B9AACE018D960E94133BA5C0B2
:108A8000F601B48081E08FA78BED88AB8AE48EA7D6
:108A9000BE016F5C7F4F8B2D0E94922CCE018D9674
:108AA0000E94133B92C0F601B4808B2D0E94B60C3D
:108AB00081E08FA78CED88ABB9AA85E08EA7CE01A7
:108AC0008D960E94133B81C0F6014481558181E05F
:108AD0008FA78DED88AB86E18EA75AAB49ABFE011F
:108AE000ED51FF4F1082FE01ED51FF4F8081982F15
:108AF0008031C8F48E010F5F1F4FBF01892F992766
:108B00009C01200F311F840F951FAA27BB27ABBFE5
:108B1000FC018791F90182ABDB018C918F5F8C9313
:108B2000982F803158F3CE018D960E94133B4DC093
:108B3000F6013496A2E8BFE080E190E021E08030C9
:108B4000920719F40E94545A03C0182E0E94545AD6
:108B500081E08FA781EE88AB84E08EA7CE018D9651
:108B60000E94133B32C081E08FA782EE88AB84E184
:108B70008EA7FE01F196A2E8BFE080E190E021E03F
:108B80008030920719F40E94435A03C0182E0E94A5
:108B9000435ACE018D960E94133B17C081E08FA7E8
:108BA00080E888AB85E08EA7F601838189ABCE0192
:108BB0008D960E94133B09C085E08EA71FA681E019
:108BC00088ABCE018D960E94133BCD51DF4F0FB67F
:108BD000F894DEBF0FBECDBFDF91CF911F910F91F3
:108BE000FF90EF90DF90CF90BF90AF900895CF931C
:108BF000DF93CDB7DEB72A970FB6F894DEBF0FBE6E
:108C0000CDBF81E08B8388E88C8384E08A83CE01AA
:108C100001960E94133B2A960FB6F894DEBF0FBE52
:108C2000CDBFDF91CF9108950F931F93CF93DF9323
:108C3000CDB7DEB7C055D0400FB6F894DEBF0FBE3B
:108C4000CDBF8A0121E02B832DE52C839E838D836C
:108C50006F8320E0261780F4AE01485F5F4F822FBC
:108C60009927DA01A80FB91FF801E80FF91F8081D1
:108C70008C932F5F261798F38FE08A83CE0101969D
:108C80000E94133BC05BDF4F0FB6F894DEBF0FBEF0
:108C9000CDBFDF91CF911F910F91089548EC50E027
:108CA00060E070E088EB9BE00E9464591092800CB9
:108CB0001092810C1092B70B0895382F2091810CDF
:108CC00088EB9BE0FC01E20FF11D30838091810C69
:108CD0008F5F8093810C8091B70B8F5F8093B70B70
:108CE0008091B70B883C18F00E944E460895809101
:108CF000810C883C10F01092810C08959091810CA9
:108D00008091800C981738F08091810C9091800CA4
:108D1000891B992708959091810C8091800C981B54
:108D2000892F8853992708952091800C88EB9BE028
:108D3000FC01E20FF11DE0818091800C8F5F809338
:108D4000800C8091B70B81508093B70B8091800C81
:108D5000883C10F01092800C8E2F992708950F9365
:108D60001F93CF93DF93EC018B0180EC0E9442486C
:108D7000015010408FEF0F3F180709F188819927A4
:108D8000803C910521F08B3D910541F00EC08BEDAB
:108D90000E9442488CED0E9442480AC08BED0E941E
:108DA00042488DED0E94424803C088810E9442489B
:108DB0002196015010408FEF0F3F1807F9F680EC15
:108DC0000E944248DF91CF911F910F9108950F9318
:108DD0001F93382F8091820C9927009719F00197E3
:108DE000C1F059C0303C09F056C01092830C20915C
:108DF000830C85E89CE0FC01E20FF11D30832F5FBE
:108E00002093830C81E08093820C84E68093840C11
:108E100042C0303C99F58091830C8230F0F0809113
:108E2000830C05E81CE0F801E80FF11D30838F5F2B
:108E30008093830C82E08093820C1092840CA801B2
:108E40006091830CC8010E945647C8010E94293BCB
:108E50001092820C1092830C1EC01092830C2091F1
:108E6000830C85E89CE0FC01E20FF11D30832F5F4D
:108E70002093830C84E68093840C0DC02091830C96
:108E800085E89CE0FC01E20FF11D30838091830CAA
:108E90008F5F8093830C8091830C893620F0109231
:108EA000820C1092830C1F910F910895FC01DA013E
:108EB00061506F3FF1F02081822F9927803C91050E
:108EC00021F08B3D910519F010C0319610C03196FC
:108ED0002081822F99278C3D910521F08D3D9105B0
:108EE00019F003C020EC01C02BED2D933196615099
:108EF00010F708958091840C882389F08091840C68
:108F000081508093840C9091840C992341F480913A
:108F1000820C813021F49093830C9093820C0895FD
:108F200085B1807F85B984B1876084B981E58CBDC6
:108F300081E08DBD08958EBD0DB407FEFDCF8EB5C9
:108F4000992708950E94FF479C9AA4988FE08093E8
:108F5000EF0CA4986A9862980895A4980895CF9306
:108F6000DF93CDB7DEB728970FB6F894DEBF0FBEFC
:108F7000CDBFA49B18C0629914C08091EE0C8530BF
:108F800050F0A4980E945A1A82E280931201109223
:108F9000380F10922F0F8091EE0C8F5F8093EE0CA4
:108FA00002C01092EE0CCE0101960E94122329817C
:108FB0003A8181E590E0289FA001299F500D389FBC
:108FC000500D1124CA01880F892F881F990B919584
:108FD0000E9400488D81882319F48F81882311F025
:108FE000A49A01C0A49828960FB6F894DEBF0FBECD
:108FF000CDBFDF91CF9108958093EF0C0895089530
:1090000008951092F10C1092F00C86E08093C2004B
:1090100088E98093C10060E875E280E090E00E94FA
:109020001C4881E08093A10F1092A20F08959093A5
:10903000F10C8093F00C08959B01AC01DC01CB0195
:10904000689412F8880F991FAA1FBB1F1694D1F7B6
:1090500080509C4DAB40BF4F689413F8220F331FD4
:10906000441F551F1694D1F7BC01CD010E94C7596A
:10907000DA01C9010197292F33272093C500809376
:10908000C4000895982F8091C00085FFFCCF909375
:10909000C60008950F931F93CF93DF938C01EB01CC
:1090A00021978FEFCF3FD80751F0F80181918F01C1
:1090B0000E9442482197FFEFCF3FDF07B1F781E0E1
:1090C00090E0DF91CF911F910F9108951F920F9221
:1090D0000FB60F9211242F933F934F935F936F938B
:1090E0007F938F939F93AF93BF93EF93FF93809161
:1090F000C6000E945D46FF91EF91BF91AF919F9195
:109100008F917F916F915F914F913F912F910F9030
:109110000FBE0F901F901895DC01FB01415050408D
:109120008FEF4F3F580741F081918D934150504050
:109130008FEF4F3F5807C1F70895DC01FB01415005
:1091400050408FEF4F3F580769F091918D918917EB
:1091500019F081E090E00895415050408FEF4F3F6B
:10916000580799F780E090E00895CF93DF93DC01F2
:10917000FB0160E0462F91E0562F8081803231F470
:10918000692F9F5F319680818032D1F3808188235F
:1091900079F08081803219F4442309F4492F8081C9
:1091A000803209F040E09F5F31968081882389F703
:1091B000442331F48081882311F4492F01C0462FC4
:1091C000262F3327E901C91BD109EC0FFD1F31966A
:1091D000842F9927821B930B01971816190624F4E4
:1091E000942F961B915001C090E091509F3F29F021
:1091F00081918D935F5F9150D8F71C925F5F852FAF
:109200009927DF91CF910895FC0190E08191882307
:1092100031F09F5F8191882311F09F3FD1F7892F13
:1092200099270895DC01FB018081882329F0819131
:109230008D9380818823D9F71C9208950F931F93F3
:10924000CF93DF93082F162FFA0141E0C0E1D7E258
:10925000C901BE010E94B4596115710581F06C9F6E
:10926000C0016D9F900D7C9F900D1124281B390B20
:10927000862F805D8193440F01E015E00AC0153010
:1092800040F0002319F080E3819302C080E28193D3
:109290004F5FC8EED3E0C901BE010E94B459611509
:1092A000710581F06C9FC0016D9F900D7C9F900DAA
:1092B0001124281B390B862F805D81934F5F01E0BD
:1092C00014E00AC0143040F0002319F080E38193C9
:1092D00002C080E281934F5FC4E6D0E0C901BE01C5
:1092E0000E94B4596115710581F04F5F6C9FC001F8
:1092F0006D9F900D7C9F900D1124281B390B862F9C
:10930000805D819301E013E00AC0133040F04F5FAD
:10931000002319F080E3819302C080E28193C901A8
:109320006AE070E00E94B4596115710591F04F5FD9
:10933000CB01880F991F880F991F880F991F860FDF
:10934000971F860F971F281B390B862F805D8193EF
:109350000AC0123040F04F5F002319F080E3819380
:1093600002C080E28193822F805D81931082842FDE
:109370009927DF91CF911F910F910895FC01262F1E
:10938000862F82958F708A3038F06AE00E94945957
:10939000892F8F5B819309C0862F82958F706AE039
:1093A0000E949459892F805D8193822F8F708A301B
:1093B00038F06AE00E949459892F8F5B808308956A
:1093C000822F8F706AE00E949459892F805D80837C
:1093D0000895EF92FF920F931F937C018B01872FCB
:1093E0009927682FC7010E94BE49C8019070682F55
:1093F000C7010E94BE491F910F91FF90EF90089501
:10940000CF92DF92EF92FF920F931F936C017A013C
:109410008B01CB01AA27BB27BC01C6010E94E949E9
:10942000D801C701A070B070BC01C6010E94E94913
:109430001F910F91FF90EF90DF90CF9008951F93B1
:10944000CF93DF93CDB7DEB768970FB6F894DEBF42
:109450000FBECDBF10E0BE016F5F7F4F812F0E9416
:10946000EB2A212F3327C901880F991F880F991FD5
:10947000880F991F820F931FFC01EE50F34F8981D3
:1094800085838A8186838B8187838C8180838D818C
:1094900081838E8182838F81838388858483888D75
:1094A0008087F901E05EF14F10821F5F143198F25E
:1094B00068960FB6F894DEBF0FBECDBFDF91CF9197
:1094C0001F9108951F93CF93DF93CDB7DEB76897B1
:1094D0000FB6F894DEBF0FBECDBF10E0A89519827D
:1094E0001A821B821C821D821E821F821886188E81
:1094F0008FE0189FC00111248059994FBC01CE0103
:1095000009960E944359BE016F5F7F4F812F0E94D1
:10951000B32A1F5F143110F368960FB6F894DEBFBC
:109520000FBECDBFDF91CF911F910895CF93C0E0C3
:1095300086E0C89FC0011124FC01E855F24FF0936A
:10954000A70DE093A60D80819181009719F00197F6
:1095500091838083E091A60DF091A70D8281938184
:10956000009719F0019793838283E091A60DF09103
:10957000A70D84819581009719F0019795838483C5
:109580002C2F3327C901880F991F880F991F880F27
:10959000991F820F931FFC01EE50F34F80818823A7
:1095A00019F48181882321F08C2F8F5D0E94E74B75
:1095B000CF5FC43108F4BCCFCF910895992787308D
:1095C000910509F466C088309105ACF484309105AA
:1095D00009F43EC08530910534F48230910511F1D3
:1095E000039759F198C08530910509F43CC006975E
:1095F00009F444C090C08A30910509F46BC08B30E7
:10960000910544F48830910509F44EC0099709F496
:1096100056C081C08B30910509F467C00C9709F4DE
:109620006FC079C080EC0E94CC39882319F081E0AA
:1096300090E0089580E090E0089581EC0E94CC399C
:10964000882319F081E090E0089580E090E008958B
:1096500082EC0E94CC39882319F081E090E00895D3
:1096600080E090E0089581ED0E94CC39882319F0C4
:1096700081E090E0089580E090E0089584EC0E94FD
:10968000CC39882319F081E090E0089580E090E0E3
:10969000089585EC0E94CC39882319F081E090E090
:1096A000089580E090E0089586EC0E94CC398823EC
:1096B00019F081E090E0089580E090E0089587EC53
:1096C0000E94CC39882319F081E090E0089580E071
:1096D00090E0089583EC0E94CC39882319F081E052
:1096E00090E0089580E090E0089582ED0E94CC39EA
:1096F000882319F081E090E0089580E090E00895DB
:1097000083ED0E94CC39882319F081E090E0089520
:1097100080E090E0089580E090E008950F93CF936B
:10972000DF93CDB7DEB721970FB6F894DEBF0FBE3B
:10973000CDBF89838150843170F000E021E0AE011B
:109740004F5F5F4F69E071E08FE591E00E94462630
:1097500080E090E007C089819927FC01E15EF14F2C
:109760008081992721960FB6F894DEBF0FBECDBF3A
:10977000DF91CF910F9108950F93CF93DF93CDB7E2
:10978000DEB721970FB6F894DEBF0FBECDBF898339
:10979000843160F000E021E0AE014F5F5F4F64E193
:1097A00071E08FE591E00E94462607C0898120E2A2
:1097B0003EE0F901E80FF11D608321960FB6F894A1
:1097C000DEBF0FBECDBFDF91CF910F910895DF9225
:1097D000EF92FF920F931F93CF93DF93CDB7DEB736
:1097E00021970FB6F894DEBF0FBECDBF198281322C
:1097F00009F46DC0823219F481E0898368C0833234
:1098000019F482E0898363C0843219F483E0898388
:109810005EC0853219F484E0898359C0863219F418
:1098200085E0898354C0873219F486E089834FC06C
:10983000883219F487E089834AC0893219F488E0B4
:10984000898345C08A3219F489E0898340C08B320C
:1098500019F48AE089833BC08C3219F48BE0898348
:1098600036C08D3219F48CE0898331C08E3219F400
:109870008DE089832CC08F3219F48EE0898327C054
:10988000803319F48FE0898322C0813319F480E199
:1098900089831DC0823319F481E1898318C0833321
:1098A00019F482E1898313C0843319F483E1898335
:1098B0000EC000E021E0AE014F5F5F4F69E471E050
:1098C0008FE591E00E94462680E090E05EC7FF248D
:1098D000EF2CDF2C298186E0289FC00111248855B8
:1098E000924F9093A70D8093A60D3327C901880F3F
:1098F000991F880F991F880F991F820F931FFC01D2
:10990000EE50F34F8081882309F4A0C18981282F6C
:109910003327C901880F991F880F991F880F991F36
:10992000820F931FFC01EE50F34F80818F3F19F49B
:10993000EE24E3948BC18981282F332702EF1CE0AA
:10994000C901880F991F880F991F880F991F820FCF
:10995000931FFC01E00FF11FE0818E2F82508B30AE
:1099600008F04CC08E2F0E94DE4A482F8981282F94
:109970003327C901880F991F880F991F880F991FD6
:10998000820F931FFC01E00FF11F808580FF02C052
:1099900081E04827442369F0E091A60DF091A70DDE
:1099A00080819181892B19F4EE24E3944FC1EE2438
:1099B0004DC1A091A60DB091A70D8981282F332705
:1099C000C901880F991F880F991F880F991F820F4F
:1099D000931FFC01EE50F34F958185E0989FC001E5
:1099E00011248D939C93E091A60DF091A70D808199
:1099F0009181019691838083EE2428C18981282F4B
:109A0000332702EF1CE0C901880F991F880F991FA7
:109A1000880F991F820F931FFC01E00FF11FE08157
:109A20008E2F8D50803208F04CC08F5F0E94B90C91
:109A3000482F8981282F3327C901880F991F880F44
:109A4000991F880F991F820F931FFC01E00FF11FD0
:109A5000808580FF02C081E04827442369F0E091BF
:109A6000A60DF091A70D80819181892B19F4EE2428
:109A7000E394ECC0EE24EAC0A091A60DB091A70D2E
:109A80008981282F3327C901880F991F880F991FB3
:109A9000880F991F820F931FFC01EE50F34F9581A1
:109AA00085E0989FC00111248D939C93E091A60DB1
:109AB000F091A70D80819181019691838083EE249E
:109AC000C5C08981282F332702EF1CE0C901880F08
:109AD000991F880F991F880F991F820F931FFC01F0
:109AE000E00FF11FE0818E2F8D52823208F04CC0C2
:109AF0008F5F0E94CC22482F8981282F3327C901EC
:109B0000880F991F880F991F880F991F820F931F25
:109B1000FC01E00FF11F808580FF02C081E0482733
:109B2000442369F0E091A60DF091A70D8081918109
:109B3000892B19F4EE24E39489C0EE2487C0A09108
:109B4000A60DB091A70D8981282F3327C901880F51
:109B5000991F880F991F880F991F820F931FFC016F
:109B6000EE50F34F958185E0989FC00111248D93AD
:109B70009C93E091A60DF091A70D808191810196B3
:109B800091838083EE2462C08981282F332702EFDE
:109B90001CE0C901880F991F880F991F880F991F12
:109BA000820F931FFC01E00FF11FE0818E2F8F5475
:109BB0008F3008F04BC08F5F0E948E4B482F8981F9
:109BC000282F3327C901880F991F880F991F880FE5
:109BD000991F820F931FFC01E00FF11F808580FF0A
:109BE00002C081E04827442369F0E091A60DF0917E
:109BF000A70D80819181892B19F4EE24E39426C06E
:109C0000EE2424C0A091A60DB091A70D8981282F24
:109C10003327C901880F991F880F991F880F991F33
:109C2000820F931FFC01EE50F34F958185E0989FC2
:109C3000C00111248D939C93E091A60DF091A70D86
:109C400080819181019691838083EE248981282FE0
:109C50003327C901880F991F880F991F880F991FF3
:109C6000820F931FFC01EE50F34F8181882311F482
:109C7000F82EA4C18981282F3327C901880F991F85
:109C8000880F991F880F991F820F931FFC01EE50B8
:109C9000F34F81818F3F19F4FF24F3948FC18981A1
:109CA000282F332702EF1CE0C901880F991F880F66
:109CB000991F880F991F820F931FFC01E00FF11F5E
:109CC0009181892F82508B3008F04DC0892F0E94DE
:109CD000DE4A482F8981282F3327C901880F991F11
:109CE000880F991F880F991F820F931FFC01E00FA7
:109CF000F11F808581FF02C081E04827442369F07D
:109D0000E091A60DF091A70D82819381892B19F422
:109D1000FF24F39453C1FF2451C1A091A60DB0912B
:109D2000A70D8981282F3327C901880F991F880F14
:109D3000991F880F991F820F931FFC01EE50F34F5C
:109D4000968185E0989FC0011124FD019383828351
:109D5000E091A60DF091A70D8281938101969383E6
:109D60008283FF242BC18981282F332702EF1CE037
:109D7000C901880F991F880F991F880F991F820F9B
:109D8000931FFC01E00FF11F9181892F8D508032CC
:109D900008F04DC08F5F0E94B90C482F8981282F91
:109DA0003327C901880F991F880F991F880F991FA2
:109DB000820F931FFC01E00FF11F808581FF02C01D
:109DC00081E04827442369F0E091A60DF091A70DAA
:109DD00082819381892B19F4FF24F394EFC0FF242F
:109DE000EDC0A091A60DB091A70D8981282F332732
:109DF000C901880F991F880F991F880F991F820F1B
:109E0000931FFC01EE50F34F968185E0989FC001AF
:109E10001124FD0193838283E091A60DF091A70D9B
:109E200082819381019693838283FF24C7C08981B5
:109E3000282F332702EF1CE0C901880F991F880FD4
:109E4000991F880F991F820F931FFC01E00FF11FCC
:109E50009181892F8D52823208F04DC08F5F0E9410
:109E6000CC22482F8981282F3327C901880F991FB9
:109E7000880F991F880F991F820F931FFC01E00F15
:109E8000F11F808581FF02C081E04827442369F0EB
:109E9000E091A60DF091A70D82819381892B19F491
:109EA000FF24F3948BC0FF2489C0A091A60DB0912C
:109EB000A70D8981282F3327C901880F991F880F83
:109EC000991F880F991F820F931FFC01EE50F34FCB
:109ED000968185E0989FC0011124FD0193838283C0
:109EE000E091A60DF091A70D828193810196938355
:109EF0008283FF2463C08981282F332702EF1CE06F
:109F0000C901880F991F880F991F880F991F820F09
:109F1000931FFC01E00FF11F9181892F8F548F3027
:109F200008F04CC08F5F0E948E4B482F8981282FEC
:109F30003327C901880F991F880F991F880F991F10
:109F4000820F931FFC01E00FF11F808581FF02C08B
:109F500081E04827442369F0E091A60DF091A70D18
:109F600082819381892B19F4FF24F39427C0FF2465
:109F700025C0A091A60DB091A70D8981282F332768
:109F8000C901880F991F880F991F880F991F820F89
:109F9000931FFC01EE50F34F968185E0989FC0011E
:109FA0001124FD0193838283E091A60DF091A70D0A
:109FB00082819381019693838283FF248981282F54
:109FC0003327C901880F991F880F991F880F991F80
:109FD000820F931FFC01EE50F34F8281882311F40E
:109FE000D82EA4C18981282F3327C901880F991F32
:109FF000880F991F880F991F820F931FFC01EE5045
:10A00000F34F82818F3F19F4DD24D3948FC189816E
:10A01000282F332702EF1CE0C901880F991F880FF2
:10A02000991F880F991F820F931FFC01E00FF11FEA
:10A030009281892F82508B3008F04DC0892F0E9469
:10A04000DE4A482F8981282F3327C901880F991F9D
:10A05000880F991F880F991F820F931FFC01E00F33
:10A06000F11F808582FF02C081E04827442369F008
:10A07000E091A60DF091A70D84819581892B19F4AB
:10A08000DD24D39453C1DD2451C1A091A60DB0911C
:10A09000A70D8981282F3327C901880F991F880FA1
:10A0A000991F880F991F820F931FFC01EE50F34FE9
:10A0B000978185E0989FC0011124FD0195838483D9
:10A0C000E091A60DF091A70D84819581019695836D
:10A0D0008483DD242BC18981282F332702EF1CE0E4
:10A0E000C901880F991F880F991F880F991F820F28
:10A0F000931FFC01E00FF11F9281892F8D50803258
:10A1000008F04DC08F5F0E94B90C482F8981282F1D
:10A110003327C901880F991F880F991F880F991F2E
:10A12000820F931FFC01E00FF11F808582FF02C0A8
:10A1300081E04827442369F0E091A60DF091A70D36
:10A1400084819581892B19F4DD24D394EFC0DD241B
:10A15000EDC0A091A60DB091A70D8981282F3327BE
:10A16000C901880F991F880F991F880F991F820FA7
:10A17000931FFC01EE50F34F978185E0989FC0013B
:10A180001124FD0195838483E091A60DF091A70D24
:10A1900084819581019695838483DD24C7C089815C
:10A1A000282F332702EF1CE0C901880F991F880F61
:10A1B000991F880F991F820F931FFC01E00FF11F59
:10A1C0009281892F8D52823208F04DC08F5F0E949C
:10A1D000CC22482F8981282F3327C901880F991F46
:10A1E000880F991F880F991F820F931FFC01E00FA2
:10A1F000F11F808582FF02C081E04827442369F077
:10A20000E091A60DF091A70D84819581892B19F419
:10A21000DD24D3948BC0DD2489C0A091A60DB0911C
:10A22000A70D8981282F3327C901880F991F880F0F
:10A23000991F880F991F820F931FFC01EE50F34F57
:10A24000978185E0989FC0011124FD019583848347
:10A25000E091A60DF091A70D8481958101969583DB
:10A260008483DD2463C08981282F332702EF1CE01B
:10A27000C901880F991F880F991F880F991F820F96
:10A28000931FFC01E00FF11F9281892F8F548F30B3
:10A2900008F04CC08F5F0E948E4B482F8981282F79
:10A2A0003327C901880F991F880F991F880F991F9D
:10A2B000820F931FFC01E00FF11F808582FF02C017
:10A2C00081E04827442369F0E091A60DF091A70DA5
:10A2D00084819581892B19F4DD24D39427C0DD2452
:10A2E00025C0A091A60DB091A70D8981282F3327F5
:10A2F000C901880F991F880F991F880F991F820F16
:10A30000931FFC01EE50F34F978185E0989FC001A9
:10A310001124FD0195838483E091A60DF091A70D92
:10A3200084819581019695838483DD244981842FDE
:10A3300099279C01220F331F220F331F220F331F37
:10A34000280F391FF901EE50F34F8081882309F45B
:10A350005AC18181882309F456C18281882309F476
:10A3600052C18381882309F077C0EE20C9F1FF2014
:10A37000B9F18481882361F46D2D842F0E94BC4B38
:10A38000DD2019F081E090E000C280E090E0FDC1A6
:10A390008981282F3327C901880F991F880F991F9A
:10A3A000880F991F820F931FFC01EE50F34F848199
:10A3B000823079F460E0ED1409F461E089810E9453
:10A3C000BC4BED1419F481E090E0DFC180E090E037
:10A3D000DCC161E089810E94BC4B81E090E0D5C185
:10A3E0004981242F3327C901880F991F880F991F8E
:10A3F000880F991F820F931FFC01EE50F34F848149
:10A40000823049F4DD2039F461E0842F0E94BC4B96
:10A4100081E090E0BAC14981842F99279C01220FE5
:10A42000331F220F331F220F331F280F391FF9014B
:10A43000EE50F34F6481613041F4DD2031F0842F20
:10A440000E94BC4B81E090E0A0C160E089810E9445
:10A45000BC4B80E090E099C14981842F99279C01F1
:10A46000220F331F220F331F220F331F280F391FD4
:10A47000F901EE50F34F8381823009F040C0EF14B0
:10A48000B9F58481882361F46D2D842F0E94BC4B23
:10A49000DD2019F081E090E078C180E090E075C1A6
:10A4A0008981282F3327C901880F991F880F991F89
:10A4B000880F991F820F931FFC01EE50F34F848188
:10A4C000823079F460E0ED1409F461E089810E9442
:10A4D000BC4BED1419F481E090E057C180E090E0AE
:10A4E00054C161E089810E94BC4B81E090E04DC184
:10A4F00060E089810E94BC4B80E090E046C1EE2084
:10A5000019F4FF2009F443C04981242F3327C901DE
:10A51000880F991F880F991F880F991F820F931F0B
:10A52000FC01EE50F34F8481882361F46D2D842F5C
:10A530000E94BC4BDD2019F081E090E026C180E054
:10A5400090E023C14981242F3327C901880F991F27
:10A55000880F991F880F991F820F931FFC01EE50DF
:10A56000F34F8481823061F46D2D842F0E94BC4BA7
:10A57000DD2019F081E090E008C180E090E005C1A5
:10A5800061E089810E94BC4B81E090E0FEC049817E
:10A59000842F99279C01220F331F220F331F220F74
:10A5A000331F280F391FF901EE50F34F64816130DA
:10A5B00041F4DD2009F1842F0E94BC4B81E090E042
:10A5C000E4C04981242F3327C901880F991F880FC0
:10A5D000991F880F991F820F931FFC01EE50F34FB4
:10A5E0008481823049F4DD2039F461E0842F0E94B7
:10A5F000BC4B81E090E0C9C060E089810E94BC4B07
:10A6000080E090E0C2C04981842F99279C01220FED
:10A61000331F220F331F220F331F280F391FF90159
:10A62000EE50F34F8081882309F44DC08181882347
:10A6300009F449C08381882391F4EE2049F0FF207A
:10A6400039F061E0842F0E94BC4B81E090E09DC016
:10A6500060E089810E94BC4B80E090E096C0498117
:10A66000242F3327C901880F991F880F991F880F3E
:10A67000991F820F931FFC01EE50F34F83818230AC
:10A6800081F4EF1439F461E0842F0E94BC4B81E027
:10A6900090E07BC060E089810E94BC4B80E090E04C
:10A6A00074C0EE2011F4FF2039F061E089810E942E
:10A6B000BC4B81E090E069C060E089810E94BC4BA6
:10A6C00080E090E062C04981842F99279C01220F8D
:10A6D000331F220F331F220F331F280F391FF90199
:10A6E000EE50F34F8181882309F44DC08281882385
:10A6F00009F449C08481882391F4EE2049F0FF20B9
:10A7000039F061E0842F0E94BC4B81E090E03DC0B5
:10A7100060E089810E94BC4B80E090E036C04981B6
:10A72000242F3327C901880F991F880F991F880F7D
:10A73000991F820F931FFC01EE50F34F84818230EA
:10A7400081F4EF1439F461E0842F0E94BC4B81E066
:10A7500090E01BC060E089810E94BC4B80E090E0EB
:10A7600014C0EE2011F4FF2039F061E089810E94CD
:10A77000BC4B81E090E009C060E089810E94BC4B45
:10A7800080E090E002C080E090E021960FB6F8945F
:10A79000DEBF0FBECDBFDF91CF911F910F91FF9014
:10A7A000EF90DF900895CF93DF93CDB7DEB7219779
:10A7B0000FB6F894DEBF0FBECDBF282F04B603FE40
:10A7C00028C0FE013196ACEBB0E081E090E031E0D2
:10A7D0008030930719F40E94435A03C0182E0E9438
:10A7E000435A8981843190F48F5F8983FE013196C9
:10A7F000ACEBB0E081E090E031E08030930719F4F9
:10A800000E94545A03C0182E0E94545A84B7877F5E
:10A8100084BF809160008861809360002093600015
:10A820008091600088608093600021960FB6F89454
:10A83000DEBF0FBECDBFDF91CF910895EF92FF92A3
:10A840000F931F937B018C0120E030E040E05FE438
:10A850000E94825688239CF020E030E040E05FECCC
:10A86000C801B7010E946C55DC01CB01BC01CD01D0
:10A870000E941C57605070408040904804C0C8013E
:10A88000B7010E941C571F910F91FF90EF90089500
:10A89000A0E0B0E0EEE4F4E50C94045A8C017B01F6
:10A8A0005A01DC018C91823058F0FB01908192308A
:10A8B00010F4A7010BC1843029F4943009F4A6C028
:10A8C000A80104C19430A9F3923009F4A9C08230E0
:10A8D00081F3F801C280D380FB0162817381F801AA
:10A8E0002481358146815781F70164807580868097
:10A8F0009780C601861B970B97FDD8C080970CF4F4
:10A900006CC06C157D050CF0ADC066247724430146
:10A91000F8016181F7018181681709F499C0662304
:10A9200009F491C0621A730A840A950AA40193017A
:10A9300057FDC0C0F5011182B60119012A01790144
:10A940008A0139014A010894610871088108910857
:10A95000FFEF6F16FFEF7F06FFEF8F06FFE39F0607
:10A96000F0F4A8019701220F331F441F551F19014E
:10A970002A01B601615070406B0179018A013901E9
:10A980004A01089461087108810891088FEF6816E0
:10A990008FEF78068FEF88068FE3980610F383E039
:10A9A000D5018C9357FC64C0F5012483358346831D
:10A9B000578373836283A50189C06F5F7F4FD40182
:10A9C000C30181709070A070B07096948794779452
:10A9D0006794682A792A8A2A9B2A6C157D056CF36C
:10A9E00011C00894C11CD11CDA01C901817090709A
:10A9F000A070B0705695479537952795282B392B21
:10AA00004A2B5B2BC616D70664F382CFF8019181DF
:10AA1000FB018181981709F453CF42E751E056C0FA
:10AA2000823009F04DCF88E0DA01F80101900D92F3
:10AA30008A95E1F7F8018181FB0191818923FA016F
:10AA40008183A50143C0261937094809590970CFE8
:10AA5000F5016183B601260D371D481D591D1901E9
:10AA60002A019DCF6B0120E030E040E050E050CF64
:10AA7000D201C101B695A7959795879521E030E061
:10AA800040E050E02222332244225522282A392A4B
:10AA90004A2A5B2AF501248235824682578208942D
:10AAA000C11CD11CD382C282A50110C09095819592
:10AAB0009F4F24CF81E0F5018183B60150954095E9
:10AAC000309521953F4F4F4F5F4F37CFCA01E2E19D
:10AAD000CDB7DEB70C94205AA0E2B0E0E2E7F5E58E
:10AAE0000C94125ADC01CB01898F9A8FAB8FBC8FEB
:10AAF0002D8F3E8F4F8F58A3BE016F5F7F4FCE01CA
:10AB000049960E9456588E01075F1F4FB801CE012B
:10AB10004D960E945658AE014F5E5F4FB801CE0170
:10AB200001960E9448540E946E57DC01CB01BC0183
:10AB3000CD01E4E0A0960C942E5AA0E2B0E0E3EA46
:10AB4000F5E50C94125ADC01CB01898F9A8FAB8FFB
:10AB5000BC8F2D8F3E8F4F8F58A3BE016F5F7F4FED
:10AB6000CE0149960E9456588E01075F1F4FB801CB
:10AB7000CE014D960E9456588A8591E089278A8792
:10AB8000AE014F5E5F4FB801CE0101960E9448545E
:10AB90000E946E57DC01CB01BC01CD01E4E0A09620
:10ABA0000C942E5AA8E1B0E0E8EDF5E50C940C5AAF
:10ABB000DC01CB01898B9A8BAB8BBC8B2D8B3E8BB5
:10ABC0004F8B588FBE016F5F7F4FCE0141960E9421
:10ABD00056588E01075F1F4FB801CE0145960E945F
:10ABE0005658FE0131962981223008F45FC039851C
:10ABF000323010F4B8017BC081819A858927818326
:10AC0000243009F455C0223009F452C0343009F41C
:10AC100054C0323009F458C06B817C818B859C858F
:10AC2000681B790B2D813E814F815885ED84FE8410
:10AC30000F8518892E153F054007510730F4220F64
:10AC4000331F441F551F615070407C836B8380E02D
:10AC500090E0A0E0B0E4AA24BB2465012E153F05D6
:10AC60004007510740F0A82AB92ACA2ADB2A2E1920
:10AC70003F09400B510BB695A79597958795220FE5
:10AC8000331F441F551F0097A105B10539F7D601A1
:10AC9000C5018F779070A070B07080349105A105C8
:10ACA000B105A9F0A482B582C682D782BF011FC0B8
:10ACB0002317E1F762E771E01AC01D821E821F822E
:10ACC00018861C821B82F2CF84E08983EFCFA7FC19
:10ACD00005C0211531054105510521F380E490E0BF
:10ACE000A0E0B0E0A80EB91ECA1EDB1EDBCFCB0170
:10ACF0000E946E57DC01CB01BC01CD01EAE06896F1
:10AD00000C94285AA8E1B0E0E8E8F6E50C94125A51
:10AD1000DC01CB01898B9A8BAB8BBC8B2D8B3E8B53
:10AD20004F8B588FBE016F5F7F4FCE0141960E94BF
:10AD300056588E01075F1F4FB801CE0145960E94FD
:10AD400056588981823018F08985823018F42FEFA7
:10AD50003FEF09C0B801CE0101960E94D058282FBC
:10AD6000332727FD3095C901E4E068960C942E5AEC
:10AD7000A8E0B0E0EEEBF6E50C94105A9B01AC01B4
:10AD80007B018C01EE2417FDE394FF24002711279B
:10AD9000EA82211531054105510539F482E08983A4
:10ADA000CE0101960E946E5743C083E089836EE115
:10ADB00070E0CB01EE2031F579018A01A8019701FD
:10ADC0002030E0E03E07E0E04E07E0E45E0798F464
:10ADD00079018A01EE0CFF1C001F111F0197BC01B5
:10ADE000A8019701E0E0EE16E0E0FE06E0E00E07C5
:10ADF000E0E41E0768F3ED82FE820F8318877C83F0
:10AE00006B83CECF2030E0E03E07E0E04E07E0E885
:10AE10005E0741F0EE24FF248701E21AF30A040BD7
:10AE2000150BCCCF7C836B8360E070E080E09FECFF
:10AE3000E6E028960C942C5AACE0B0E0E2E2F7E5AC
:10AE40000C94145ADC01CB0189879A87AB87BC87A5
:10AE5000BE016F5F7F4FCE0109960E9456588981CF
:10AE6000823011F0823028F460E070E080E090E001
:10AE700031C0843039F02B813C8137FDF5CF2F3143
:10AE800031056CF08A81882329F060E070E080E071
:10AE900090E820C06FEF7FEF8FEF9FE71BC08EE140
:10AEA00090E0821B930B2D813E814F81588504C019
:10AEB00056954795379527958A95D2F78A818823A5
:10AEC00039F050954095309521953F4F4F4F5F4F4A
:10AED000CA01B901E2E02C960C94305AA0E0B0E02F
:10AEE000E4E7F7E50C940A5A882499245401DC011C
:10AEF000FC0124813581468157818181082F1127EA
:10AF000060E070E08C91823020F46FEF70E040617F
:10AF1000A4C0843009F464C0823009F463C02115F0
:10AF200031054105510509F498C0FD0182819381E5
:10AF3000FFEF82389F070CF050C0A2E8EA2EAFEF77
:10AF4000FA2EE81AF90A8AE1E816F1040CF06BC04F
:10AF50006B0181E090E0A0E0B0E00E2C04C0880F0F
:10AF6000991FAA1FBB1F0A94D2F70197A109B10923
:10AF700082239323A423B5230097A105B10519F0DB
:10AF8000F1E0CF2ED12C04C05695479537952795E3
:10AF9000EA94D2F7C601AA2797FDA095BA2F282BCD
:10AFA000392B4A2B5B2BDA01C9018F779070A07087
:10AFB000B07080349105A105B105D1F1215C3F4FFE
:10AFC0004F4F5F4F2030E0E03E07E0E04E07E0E407
:10AFD0005E0708F161E070E01EC0803891053CF02A
:10AFE0006FEF70E020E030E040E050E036C0BC01A0
:10AFF00061587F4FDA01C9018F779070A070B070EF
:10B0000080349105A105B105D1F0215C3F4F4F4F30
:10B010005F4F57FD1BC097E056954795379527958D
:10B020009A95D1F71AC020E030E040E050E0BBCF65
:10B0300027FFC8CF205C3F4F4F4F5F4FC3CF27FF45
:10B04000E8CF205C3F4F4F4F5F4FE3CF569547957A
:10B05000379527956F5F7F4FDECF822E932E942FEB
:10B060009F778A2D8078A82EA92A962F97959927C1
:10B0700097958A2D8F77A82EA92A76956795962F72
:10B080009F778B2D8078B82EB92A902F9795992786
:10B0900097958B2D8F77B82EB92AD501C401BC01A5
:10B0A000CD01ECE0CDB7DEB70C94265ACF93DF93F9
:10B0B000FC01DB01408151812281622F6F7770E0BA
:10B0C000221F2227221F9381892F880F822B282F4E
:10B0D0003327991F9927991FED0199832115310570
:10B0E00041F44115510561057105E1F482E08C934D
:10B0F00054C02F3F310509F441C02F573040FD01A6
:10B100003383228383E08C9387E0440F551F661FAF
:10B11000771F8A95D1F77064ED014C835D836E8350
:10B120007F833BC022E83FEFF901C7E0440F551F82
:10B13000661F771FCA95D1F783E08C93403080E07B
:10B14000580780E0680780E4780778F4440F551FBB
:10B15000661F771F21503040F9014030C0E05C0786
:10B16000C0E06C07C0E47C0788F3ED01FB83EA8351
:10B17000FD0144835583668377830FC041155105D4
:10B180006105710519F484E08C9307C064FF03C066
:10B1900081E08C93C1CF1C92BFCFDF91CF910895F6
:10B1A0000F931F93CF93DF93FC01DB0180818230EB
:10B1B00018F09C91923018F461E070E05EC0843029
:10B1C000C1F0843001F1943009F447C0823009F4B1
:10B1D0004BC0823009F44EC09230A9F04181ED019C
:10B1E00089814817B9F0442389F08FEF9FEFBC01A4
:10B1F00044C0943031F7EB018981682F7727818132
:10B20000681B71093AC08181882379F781E090E059
:10B21000BC0133C022813381ED018A819B81821779
:10B2200093070CF3281739079CF0048115812681B8
:10B230003781FD016481758186819781601771076F
:10B240008207930780F2061717072807390778F453
:10B25000442359F281E090E0DBCFFD018181882316
:10B2600021F281E090E0D4CF923009F0B2CF60E0DB
:10B2700070E003C0ED018981F2CFCB01DF91CF9166
:10B280001F910F910895FB01DC0105900D920020A4
:10B29000E1F70895FB01DC0104C08D910190801954
:10B2A00021F441505040C8F7881B990B0895FB01C9
:10B2B000DC0140FF05C002C001900D9201900D928B
:10B2C00042505040C8F70895DC0140FF03C001C060
:10B2D0006D936D9342505040D8F70895FB01DC0107
:10B2E00001900D920020E1F70895629FD001739FB5
:10B2F000F001829FE00DF11D649FE00DF11D929F12
:10B30000F00D839FF00D749FF00D659FF00D992750
:10B31000729FB00DE11DF91F639FB00DE11DF91F74
:10B32000BD01CF0111240895991B79E004C0991F34
:10B33000961708F0961B881F7A95C9F7809508958F
:10B34000AA1BBB1B51E107C0AA1FBB1FA617B7074B
:10B3500010F0A61BB70B881F991F5A95A9F7809567
:10B360009095BC01CD01089597FB092E07260AD0C0
:10B3700077FD04D0E5DF06D000201AF470956195C2
:10B380007F4F0895F6F7909581959F4F0895A1E21C
:10B390001A2EAA1BBB1BFD010DC0AA1FBB1FEE1F4F
:10B3A000FF1FA217B307E407F50720F0A21BB30B9A
:10B3B000E40BF50B661F771F881F991F1A9469F716
:10B3C00060957095809590959B01AC01BD01CF0172
:10B3D000089597FB092E05260ED057FD04D0D7DF20
:10B3E0000AD0001C38F450954095309521953F4F78
:10B3F0004F4F5F4F0895F6F7909580957095619542
:10B400007F4F8F4F9F4F08952F923F924F925F92A1
:10B410006F927F928F929F92AF92BF92CF92DF9264
:10B42000EF92FF920F931F93CF93DF93CDB7DEB7C9
:10B43000CA1BDB0B0FB6F894DEBF0FBECDBF09945D
:10B440002A88398848885F846E847D848C849B84B4
:10B45000AA84B984C884DF80EE80FD800C811B81C2
:10B46000AA81B981CE0FD11D0FB6F894DEBF0FBEF1
:10B47000CDBFED010895F999FECFB2BDA1BDF89AF7
:10B48000119600B40895F7DF01921A94E1F7089538
:10B49000F999FECFB2BDA1BD00BC11960FB6F894CC
:10B4A000FA9AF99A0FBE08950190F2DF1A94E1F723
:02B4B0000895FD
:10B4B20001012E2E2F63616E5F696E7075742E63AB
:10B4C200006E222E2E2F6368616E6E656C732E6382
:10B4D20000455233002E2E2F656570726F6D6368C2
:10B4E200616E6E656C732E630050434D30004552A1
:10B4F20033004C4F4730340050434D207665722064
:10B50200392E3130004F425220383434300B002E65
:10B512002E2F7669727475656C5F696E7075742E04
:0AB5220063000000000000000000BC
:00000001FF
